:020000040040BA
:10000000B84B0020656440006164400061644000BA
:1000100061644000616440006164400000000000D1
:100020000000000000000000000000000168400027
:10003000616440000000000061684000C568400045
:10004000616440006164400061644000616440009C
:100050006164400061644000616440000000000091
:10006000616440007D80400000000000C940400005
:10007000DD404000715C400061644000616440000C
:100080006164400061644000815C4000D920400010
:10009000918040006164400061644000310A40008A
:1000A000616440006164400061644000616440003C
:1000B00061644000150940006164400000000000D8
:1000C0000000000000000000000000000000000030
:1000D0000000000000000000000000000000000020
:1000E0000000000000000000000000000000000010
:1000F00000000000000000000000000061644000FB
:10010000DD5140006164400000000000000000007C
:1001100000000000000000000000000000000000DF
:1001200000000000000000000000000000000000CF
:1001300000000000000000000000000000000000BF
:10014000000000000000000010B5054C237833B912
:10015000044B13B10448AFF300800123237010BD9A
:10016000B80B002000000000D0C340000C4B43B18E
:100170000C480D4910B5AFF300800C48036823B953
:1001800010BD0A48036833B97047094B002BF7D0FC
:10019000BDE810401847064B002BF5D0184700BFAC
:1001A00000000000D0C34000BC0B0020D0C34000C2
:1001B0000000000030B587B01D20184B9847184C40
:1001C000236C23F4001323646846164B9847694652
:1001D0002046154B984704232361082323610123FC
:1001E0002361626822F08F026260104A0321204678
:1001F0000F4DA847002120460E4B9847636813F027
:10020000800F01D1082222600B4B4FF000521A6080
:10021000702283F81D2307B030BD00BFA9614000E4
:100220000080034001084000950840005D02400046
:10023000E50840002908400000E100E00222014BEF
:100240001A60704700800340024B1880024B1980EF
:10025000704700BF820000208400002010B5064CCB
:10026000206D80B2054B9847A06DE16D89B280B2D8
:10027000034B984710BD00BF008003404D2840004D
:1002800049024000014B1888704700BF82000020DF
:10029000014B1888704700BF840000200D4B1B885D
:1002A00040F68962934205D90B4A12883E2A01D84A
:1002B00003207047084A128840F689618A4203D9B0
:1002C0003E2B01D804207047934201D8022070478A
:1002D0000120704782000020840000200120704728
:1002E0007047012070470020704770470120704719
:1002F000014B1878704700BFDC0B002070470000EE
:1003000058B908B5054B1B78012B00D008BD044B2C
:100310001B68002BFAD09847F8E77047E00B0020E5
:10032000D40B002008B50C4B9847C3780B4A1370C8
:10033000012B0CD101220A4B1A700022094B1A80A2
:10034000094B9847094B1B681BB1984701E0084BC4
:100350009847012008BD00BF253D4000DC0B002070
:10036000E00B0020DE0B002061804000D40B002059
:100370006D80400008B5054B1B78012B00D008BDEF
:100380000022034B1A70034B9847F8E7DC0B002060
:10039000E00B00206D80400010B582B0074B009349
:1003A0000B46024600218420054CA04718B9054A97
:1003B00013680133136002B010BD00BF0103400099
:1003C00079584000D80B0020014B1860704700BFDF
:1003D000D40B00202DE9F0474FF40046BF4B5E6080
:1003E0000B20BF4CA0470C20A047BE4B4FF0400C49
:1003F000C3F810C0C3F8A0C0C3F834C04FF0807E6B
:10040000C3F810E0C3F8A0E0C3F834E0B64A01270F
:100410001761C2F8A070576302241461C2F8A040AB
:1004200054631C61C3F8A0405C631F66C3F89070FE
:100430005F655F62C3F88070196F39431967596F40
:1004400021F0010159675F604FF480311966C3F8EC
:10045000901059655962C3F88010186F08431867E7
:10046000586F20F48030586759601C61C3F8A04071
:100470005C6304205861C3F8A0005866C3F890007C
:1004800058655862C3F88000196F21F0040119679C
:10049000596F21F00401596718211966C3F89010AB
:1004A00059655962C3F880101D6F25F018051D6746
:1004B0005D6F25F018055D67596008251D66C3F856
:1004C00090505D655D62C3F88050196F21F008019E
:1004D0001967596F21F0080159675D60102119668D
:1004E000C3F8901059655962C3F88010D3F8708032
:1004F00028F01008C3F87080D3F8748028F0100832
:10050000C3F8748059604FF48028C3F81480C3F88E
:10051000A0804FF02009C3F81490C3F8A090C3F84E
:1005200010C0C3F8A0C0C3F834C0C3F810E0C3F8CB
:10053000A0E0C3F834E01761C2F8A07057631461FB
:10054000C2F8A04054634FF4007CC3F860C0C3F805
:1005500090C0C3F854C0C3F824C0C3F880C01C6F57
:1005600044EA0C041C675C6F24F400745C67C3F8F5
:1005700004C04FF480641C66C3F890405C655C6204
:10058000C3F880401F6F27431F675F6F27F48067A2
:100590005F675C604FF4006EC3F810E0C3F8A0E042
:1005A000C3F834E04FF400275F61C3F8A0701F6602
:1005B000C3F890705F655F62C3F880701F6F27F4A7
:1005C00000271F675F6F27F400275F674FF48017CE
:1005D0005F61C3F8A0701F66C3F890705F655F62CB
:1005E000C3F880701F6F27F480171F675F6F27F4B1
:1005F00080175F674FF480575F61C3F8A0705F6634
:10060000C3F890705F655F62C3F880701F6F27F456
:1006100080571F675F6F27F480575F674FF400575D
:100620005F61C3F8A0704FF480775761C2F8A07083
:100630004FF48048C3F86080C3F89080C3F85080BE
:10064000C3F82480C3F88080D3F870A02AF4804ACD
:10065000C3F870A0D3F874A02AF4804AC3F874A039
:10066000C3F81080C3F8A080C3F830805E61C3F87F
:10067000A0604FF400365E61C3F8A0601066C2F857
:10068000900050655062C2F88000166F26F0040694
:100690001667566F26F00406566750601566C2F856
:1006A000905055655562C2F88050106F20F00800D8
:1006B0001067506F20F00800506755600B4DD5F85B
:1006C000140140F03000C5F814015161C2F8A010C7
:1006D0005166C2F890105165516209E050140E4005
:1006E000A9614000000E0E4000100E4000020E40B6
:1006F000C2F88010116F21F010011167516F21F0C5
:1007000010015167C2F81090C2F8A090C2F834905E
:10071000C2F810C0C2F8A0C0C2F830C04FF4000147
:100720005961C3F8A0105966C3F890105965596211
:10073000C3F88010196F21F400011967596F21F473
:1007400000015967C2F860E0C2F890E0C2F854E0D6
:10075000C2F824E0C2F880E0116F21F40061116753
:10076000516F21F400615167C2F804E01466C2F8C9
:10077000904054655462C2F88040116F21F480614A
:100780001167516F21F48061516754601F66C3F88F
:1007900090701F655F62C3F880701A6F22F48072D8
:1007A0001A675A6F22F480725A671F61C3F8A070EB
:1007B0001F63BDE8F08700BF08B5034B53F8203036
:1007C00003B1984708BD00BFC40E002010B582B029
:1007D000036B0193002400E00134172C09D8064B69
:1007E00053F82420019B1A42F6D02046034B984729
:1007F000F2E702B010BD00BFECBD4000B9074000F9
:1008000000230360064A4260064A82604FF4802259
:10081000C2600222027442748374C3740375704709
:100820000000DC05808D5B00036C19430164704798
:1008300010B58B7C23B34FF000434A688C6864008A
:10084000B2FBF4F2013A120292B213430A7C12068E
:1008500002F0706213434A7C120702F040521343C5
:10086000CA6813434360CB7C63B14FF080730A7D49
:1008700052B90022134303640968054B984710BD21
:100880000023DAE70023F2E74FF48012F2E700BF1B
:100890002908400008B5036B13F0807F01D01920B0
:1008A00008BD01230360064B9847002304E00021A4
:1008B000044A42F823100133172BF8D9002008BD51
:1008C00031084000C40E0020B1F1FF3F04D0044BBA
:1008D00053F82130436270474FF0FF334362704753
:1008E000ECBD400010B5084C44F82120074A4FF0F9
:1008F0000054C2F880411B01DBB282F81D33146042
:10090000034B984710BD00BFC40E002000E100E07B
:10091000C908400008B50248024B984708BD00BF0F
:1009200000800340CD07400010B51720234CA0479E
:100930001820A047224B4FF480321A66C3F890204B
:100940005A655A62C3F88020196F11431967596FAD
:1009500021F4803159675A6001225A66C3F8902009
:100960005A655A62C3F88020196F11431967596F8D
:1009700021F0010159675A60A3F5206340F2126229
:10098000DA644FF400621A600E4B0F4A5A6041223B
:100990005A62052119600D4A5A644FF4F572DA65FE
:1009A00000229A6519640A4B1A700A4B4FF4000230
:1009B0001A60702283F8172310BD00BFA9614000A0
:1009C000000E0E40000001400406090001C4000AA8
:1009D000280F002000E100E0642800D964200F4ABD
:1009E000D36D03FB00F30E49A1FB03135B09936571
:1009F00048B10A4B5A6C22F040625A645A6C42F079
:100A000080625A6470471346526C22F040625A6406
:100A10005A6C42F000625A64704700BF0000014007
:100A20001F85EB51014B1888704700BF2C0F002029
:100A30000F4B1B6A13F0010F06D000220D490A70FC
:100A40000D490A600D490A6013F0400F0ED00122D3
:100A5000084B1A70064B9A69094BB3FBF2F3064A2E
:100A60001360C3EB03139A00044B1A60704700BF76
:100A700000000140280F0020240F00202C0F002030
:100A80001F1A0500014B1870704700BFB00000200E
:100A9000064B1B7823B94FF40062054B1A6370476D
:100AA0004FF40062024B5A63704700BFB000002051
:100AB000000E0E40064B1B7823B94FF40062054B25
:100AC0005A6370474FF40062024B1A63704700BFCD
:100AD000B0000020000E0E402DE9F04186B088469F
:100AE00016461F46D0B9244B984705460024049467
:100AF00098238DF8043001238DF8053002238DF8FA
:100B0000063003238DF8083005AB03938DF807807A
:100B10008DF815402846194B984705E0184B984723
:100B20000546E3E70134E4B2B4421ED28DF8144026
:100B30003B5D8DF81630322201A92846114B9847AB
:100B4000AB79DBB2022BEDD028460F4B984732220F
:100B500001A928460B4B9847AB79DBB2022BE1D0B9
:100B600028460A4B9847002003E02846074B984741
:100B7000012006B0BDE8F0815180400045254000CD
:100B800059804000712540001D2740005925400034
:100B90002DE9F04186B00F4616469846B8B9344B59
:100BA000984704460025049598238DF804300123C6
:100BB0008DF805308DF8065002238DF8083005AB0E
:100BC00003938DF8075020462A4B98470EE02A4B96
:100BD00098470446E6E72046284B9847002044E023
:100BE0009DF8153008F805300135EDB2B54238D220
:100BF0008DF814708DF8155000238DF806303222D0
:100C000001A920461E4B9847A379DBB2022B0BD0DB
:100C100020461C4B9847322201A92046184B984782
:100C2000A379DBB2022BD6D101238DF80630322214
:100C300001A92046124B9847A379DBB2022BCFD0F3
:100C40002046104B9847322201A920460C4B98476A
:100C5000A379DBB2022BC3D02046084B9847002073
:100C600003E02046054B9847012006B0BDE8F0811F
:100C700051804000452540005980400059254000E2
:100C8000712540001D27400070B506460C46104BEC
:100C9000AA221A7011225A700222F0210D4DA84783
:100CA000012801D0002070BD220AE4B2084B1A705E
:100CB0005C709A70DC701A715C7100229A719022DB
:100CC000DA7102221A720922C2213046A84770BD89
:100CD000300F0020D90A400010B50022054B1A70D1
:100CE00029B91121034B0122034CA04710BD10214B
:100CF000F8E700BF300F0020D90A400010B50022ED
:100D0000054B1A7029B92821034B0122034CA04737
:100D100010BD2921F8E700BF300F0020D90A40009C
:100D200010B539B90022044B1A7001223621034C48
:100D3000A04710BD0322F6E7300F0020D90A40007B
:100D400038B505460C4BAA221A7012225A7002229C
:100D5000F0210A4CA047012801D0002038BD064BE5
:100D60000322BF212846064CA047012801D00020BD
:100D700038BD014B987838BD300F0020D90A4000AB
:100D8000910B400010B50B462C227021014CA0475E
:100D900010BD00BFD90A40002DE9F04182B0002308
:100DA0008DF80730012906D002291ED1114D804649
:100DB000012000240BE0104DF9E70DF10703024676
:100DC00040460E4EB0473C44E4B20134E4B2012840
:100DD0000CD123462F5D4FB1621CA95C012FECD9C9
:100DE00002332B44781EC0B2E9E7002002B0BDE810
:100DF000F08100BF4CBE400004BF4000D90A400053
:100E000010B51B4B00221A725A729A724FF4487135
:100E100099806421D9801A805A80164B9847012105
:100E2000154B9847012802D0114B187A10BD0122AA
:100E30000F4B1A720F4B98470521104B98470346EA
:100E400050B10B4A5372002BEED00A4B98470C4B13
:100E50009847074B5880E7E7064CA0470021064B10
:100E60009847A0470321054B98470346E9E700BF91
:100E7000700F002059804000FD0E4000111140000D
:100E8000A1104000014B187A704700BF700F00207E
:100E900008B5114B1B7A6BB90F4B9B7A8BB10E4A7D
:100EA00011889388D2889B1A994214DC00220A4B3D
:100EB0009A7208BD094B9847094B9847064B188012
:100EC000EAE7054A11889388D2881344994202DBE5
:100ED0000122014B9A7208BD700F0020598040001A
:100EE00031104000014B987A704700BF700F00200E
:100EF000014B1888704700BF700F002030B587B0D5
:100F000005460C4600238DF8073072228DF8082024
:100F10008DF80B3001228DF809208DF80C200DF191
:100F20000702049202228DF80A2005933C4B984751
:100F3000322202A928463B4B9847002C3BD1012482
:100F400002238DF80A3080238DF80B3001238DF8B1
:100F500007309C423CD08F238DF80B3003238DF853
:100F60000A30012C3BD09DF8073003F0F00343F02A
:100F700002038DF8073002238DF80A30012C35D09A
:100F800007238DF80730F9238DF80B30012C34D06E
:100F900005238DF8073080238DF80B30012C33D0DA
:100FA0002846214B9847012C35D000221F4B1A7040
:100FB000204607B030BDA8238DF80B3001238DF8F3
:100FC0000730322202A92846164B98470446B7E755
:100FD000322202A92846134B98470446BBE7322227
:100FE00002A928460F4B98470446BCE7322202A9C3
:100FF00028460C4B98470446C2E7322202A92846ED
:10100000084B98470446C3E7322202A92846054BFD
:1010100098470446C4E70122044B1A70C8E700BF92
:10102000452540007125400059254000E10B002076
:1010300030B587B004460023059301AB04937223B7
:101040008DF8083001238DF809309C238DF80B3082
:1010500002238DF80C3003238DF80A300C4B98478F
:10106000322202A920460B4B9847054620460A4BE0
:101070009847012D04D00020084B187007B030BDF0
:101080009DF804009DF8053000EB032080B2F5E7E1
:10109000452540007125400059254000E10B002006
:1010A00030B587B004460023059301AB0493722347
:1010B0008DF8083001238DF80930C0238DF80B30EE
:1010C00002238DF80C3003238DF80A300C4B98471F
:1010D000322202A920460B4B9847054620460A4B70
:1010E0009847012D04D00020084B187007B030BD80
:1010F0009DF804009DF8053000EB032080B2F5E771
:10110000452540007125400059254000E10B002095
:10111000F0B587B00646002305930DF1070304934D
:1011200072238DF8083001248DF80940D9238DF8F9
:101130000B308DF80C4002238DF80A304901C9B2FA
:1011400041F010018DF80710204B9847322202A978
:1011500030461F4B98470546D7238DF80B308DF846
:101160000740A0420BD030461A4B9847DC238DF83D
:101170000B3003238DF80A300024274608E0322282
:1011800002A93046124B98470546ECE70134A4B259
:10119000012D18D1BFB9092C15D819200E4B98472D
:1011A00030460A4B9847322202A93046084B9847EE
:1011B00005463046074B98479DF8073013F0010F5E
:1011C000E4D00127E2E7384607B0F0BD45254000EE
:1011D000712540005925400055744000F0B587B096
:1011E00004460E46234B9847002304938A238DF828
:1011F000043001238DF805308DF808300DF1170308
:10120000039334278DF8077002238DF80630337866
:101210008DF81730322201A92046174DA8478DF8C6
:10122000077033788DF81730322201A92046A8477D
:101230008DF8077033788DF81730322201A92046D7
:10124000A84735238DF8073073788DF81730322290
:1012500001A92046A84736238DF80730B3788DF8CA
:101260001730322201A92046A8472046034B984751
:1012700007B0F0BD452540007125400059254000CC
:10128000F0B587B00446002505958A238DF808300F
:1012900001268DF809608DF80C600DF107030493A9
:1012A0002B4B984755238DF807308DF80B500223B0
:1012B0008DF80A30322202A92046264DA847032382
:1012C0008DF807308DF80B60322202A92046A8471E
:1012D0008DF8076004238DF80B30322202A92046D6
:1012E000A84707238DF8073030238DF80B303222C2
:1012F00002A92046A8470F278DF8077031238DF8E3
:101300000B30322202A92046A8478DF807703226FA
:101310008DF80B60324602A92046A8478DF8077069
:1013200033238DF80B30324602A92046A8472046C9
:10133000094B9847094B1B68ADF804301B0C8DF81E
:10134000063001A92046064B984707B0F0BD00BF04
:101350004525400071254000592540009CBF4000B4
:10136000DD11400030B587B0054610238DF80830F8
:101370002022554B1A630A20544B98472846544B59
:10138000984700230593E7238DF80B300DF10703F1
:10139000049301238DF80C308DF8093003238DF868
:1013A0000A30322202A928464A4B984704469DF843
:1013B000073043F001038DF8073002238DF80A301F
:1013C000012842D006238DF80B3003238DF80A3014
:1013D000012C41D09DF8073063F07F038DF8073072
:1013E00002238DF80A30012C3DD000238DF8073000
:1013F0000C238DF80B30012C3CD00D238DF80B30D5
:10140000012C3ED00E238DF80B30012C40D00F2341
:101410008DF80B30012C42D0E7238DF80B300323DD
:101420008DF80A30012C41D09DF8073023F00103DC
:101430008DF8073002238DF80A30012C3DD0284664
:10144000254B9847204607B030BD322202A92846D6
:10145000204B98470446B5E7322202A928461D4B87
:1014600098470446B6E7322202A92846194B984706
:101470000446BAE7322202A92846164B984704468A
:10148000BBE7322202A92846124B98470446B9E727
:10149000322202A928460F4B98470446B7E732226A
:1014A00002A928460B4B98470446B5E7322202A909
:1014B0002846084B98470446B6E7322202A9284638
:1014C000044B98470446BAE700100E40557440009C
:1014D00045254000712540005925400030B587B0B2
:1014E00004460D4600220592A8238DF808300123FA
:1014F0008DF809308DF80B200DF1070204928DF85C
:101500000C3002238DF80A30124B9847012D0ED073
:10151000022D15D000238DF80730322202A9204673
:101520000D4B984720460D4B984707B030BD03231D
:101530008DF80730322202A92046074B9847F1E781
:1015400002238DF80730322202A92046024B984729
:10155000E8E700BF452540007125400059254000BF
:1015600030B587B072238DF8003001238DF801303B
:1015700000238DF802308DF8033008228DF8042006
:1015800004AA029203938DF81000C0F307238DF88C
:101590001130C0F307438DF81230000E8DF81300A0
:1015A0008DF81410C1F307238DF81530C1F30743EC
:1015B0008DF81630090E8DF81710084CA047084B0F
:1015C0009847A04732226946064B98470546A047F0
:1015D000054B9847284607B030BD00BF51804000FA
:1015E00045254000712540005925400030B587B0A1
:1015F0000D4672238DF8043001238DF80530002349
:101600008DF806308DF8073004228DF8082005AAE1
:10161000039204938DF81400C0F307238DF815305E
:10162000C0F307438DF81630000E8DF81700184CE4
:10163000A047184B9847A047322201A9164B98475C
:101640000446012808D0124B9847144B9847012CA8
:101650000DD0204607B030BD01238DF806300C4B6D
:101660009847322201A90C4B98470446EBE79DF8B6
:1016700014309DF8152003EB02239DF8162003EB90
:1016800002439DF8172003EB02632B60E1E700BFE4
:1016900051804000452540007125400059254000FB
:1016A0002DE9F04383B080460F4691461BB11E469C
:1016B000002501201CE0012001282BD0012833D077
:1016C000012836D0012839D04FF4000301930824B3
:1016D0003FE0EA18B25C4FEAC30E02FA0EF2114480
:1016E0000133DBB2A342F4D301280CD02544EDB280
:1016F000AC46BD42E0D27C1B042C28BF0424E4B2DB
:1017000000231946EEE70CF1201000F580701A4B0B
:101710009847EBE74FEA084101F4FE0101F50001AB
:101720001648154B9847C9E739461548124B984754
:10173000C6E749461348104B9847C3E7F2211248C1
:101740000D4B9847C0E701A90C48104B9847013C46
:10175000E4B2012804D11CB1019B13F4000FF2D1B3
:1017600018B9052003B0BDE8F0830CB90620F9E7ED
:101770009DF80700F6E700BF61154000100120004A
:101780001801200014012000FC002000ED1540008D
:1017900010B582B0094B93E8030000908DF8041057
:1017A0006B46002205210120054CA047034610B9D5
:1017B0000121044A1170184602B010BDA0BF4000BC
:1017C000A1164000E20B002038B50D46002302466A
:1017D00004213120064CA047044608B1204638BDFC
:1017E00029460448044B98470128F7D00524F5E71B
:1017F000A116400020012000ED15400010B582B078
:101800008DF804100B0A8DF805300B0C8DF806309E
:10181000090E8DF8071001AB024604212120024C6D
:10182000A04702B010BD00BFA116400008B5044B90
:101830001B780BB1002008BD024B984708BD00BFC4
:10184000E20B0020911740002DE9F04383B059B11D
:10185000012904D00124204603B0BDE8F08340F6FE
:101860005D0740F6050503E040F2DD7740F285753F
:1018700080464FF000094C4601E0002CEBD1BD4200
:10188000E9D225F00306002CF7D101A93046164B0A
:10189000984704460028F0D1019B8DF80030C3F32F
:1018A00007228DF80120C3F307428DF802201B0E9A
:1018B0008DF80330E9B2F3B2C91AC9B2C1F1040319
:1018C000BE1B9E4228BF1E46042E28BF0426F6B229
:1018D0003246694408EB0900044B984735444E44AE
:1018E0005FFA86F9C9E700BFC9174000D1944000EC
:1018F00028B1012801D000207047094800E00948BC
:1019000000B583B001A9084B984728B9019B13F48F
:10191000006F02D0012000E0002003B05DF804FB5E
:101920004000350040003100C917400010B52DEDD2
:10193000028B82B0044601A93548364B98470346CE
:10194000F8B14BB3002B32D0002B3BD0DFED328A05
:10195000002B49D09FED308A73B9DDED017AB8EEE6
:10196000677AC8EE077A9FED2D7A67EE877AFCEEEC
:10197000E77A17EE902A6281184602B0BDEC028B1E
:1019800010BD02A951F8043D23801B0C638024483C
:10199000204B98470346D4E702A951F8043DA380A1
:1019A0001B0CE3801F481B4B98470346CAE702A95C
:1019B00051F8043D03F01F0323721B48154B984751
:1019C0000346C1E702A951F8043DC3F3094308EEF9
:1019D000903AF8EE688A9FED158A68EE888A144876
:1019E0000C4B98470346B3E702A951F8043DDBB21C
:1019F00008EE103AB8EE488A28EE888ADFED077ABA
:101A000028EE278A0B48034B98470346A4E700BFFC
:101A100030082200C9174000000000000000C84242
:101A200038082200540822000800200000401C460C
:101A3000040822001408220010B582B0802300930D
:101A4000054B152214210548054CA04710B1002074
:101A500002B010BD0120FBE77C0F0020000A0E4001
:101A60000100002008B5002213210348034B9847CA
:101A7000B0FA80F0400908BD000A0E40095F40003E
:101A800010B5EFF3108404B972B6002308E09A0091
:101A900002F580020A4951F82310116001339BB20C
:101AA0007F2BF4D9002212210648074B9847C0B279
:101AB00004B962B608B1002010BD012010BD00BFFE
:101AC0007C0F0020000A0E40095F400010B4002483
:101AD0000EE0400080F00700C0B20133DBB2072BFC
:101AE00005D810F0800FF4D14000C0B2F5E7013402
:101AF000944204D211F8013B58400023EFE75DF80F
:101B0000044B704708B5094B1B781BB1022B01D061
:101B1000074808BD074B9847012804D10122034B11
:101B20001A70034808BD002008BD00BFE30B002069
:101B30007C0F0020391A400008B5094B1B781BB1F7
:101B4000022B01D0074808BD074B9847012804D154
:101B50000122034B1A70034808BD002008BD00BFD6
:101B6000E30B00207C0F0020391A4000A8B108B513
:101B70000346B1F5007F12D28818B0F5007F01D975
:101B8000002008BD08461946064B1844064B9847E6
:101B90000222064B1A70012008BD00207047002069
:101BA00008BD00BF7C0F0020D1944000E30B002053
:101BB00008B5064B1B78022B01D0002008BD044B52
:101BC00098470128FAD1034B984708BDE30B002042
:101BD000651A4000811A400090B110B504460268B1
:101BE000094B9A4201D0002010BD9A220146FF20E5
:101BF000064B984794F89A30984203D0002010BDC5
:101C000000207047012010BD5FE1AD5ACD1A4000A1
:101C10002DE9F84305460E4617460A469C211E4B01
:101C200098470446451B40B1731B052B05D94378E3
:101C3000552B07D010237B7001E000237B702046DA
:101C4000BDE8F88390F80280C37888EA0303FF2B8D
:101C500002D011237B70F2E790F80490437909EBEE
:101C600003291FFA89F9B9F13A0F06D84D44063510
:101C7000AE4205D200237B70E1E712237B70DEE7E2
:101C80004A46811D381D054B9847A7F8029087F8F2
:101C9000008001237B70D2E731944000D194400052
:101CA00010B553889C1D8C4219D83A2B01D90020BD
:101CB00010BD11469C230370552343701378837025
:101CC0001378DB43C3709378037153881B0A437105
:101CD000528804310630034B9847012010BD002084
:101CE00010BD00BFD194400070B582B004460378A7
:101CF0004C3B0C2B00F2A780DFE803F007A5A5A55D
:101D0000A5A5A5A5A52476518E004388032B05D053
:101D1000504B00225A8082221A7099E003798DF884
:101D2000043043798DF8053083798DF806304A4BBD
:101D3000984701A9494B9847464B00225A80812277
:101D40001A7085E04388012B05D0424B00225A804F
:101D500082221A707CE003790F2B05D93D4B0022BB
:101D60005A8082221A7073E03D4B9847394A5523B6
:101D7000137020235380237900EB431006684568D5
:101D80008468C16856609560D460116106694569D0
:101D90008469C16956619561D461116258E04388D4
:101DA000212B05D02B4B00225A8082221A704FE043
:101DB00001790F2905D9274B00225A8082221A70F7
:101DC00046E0202249010530264B9847012805D0DE
:101DD000204B00225A8082221A7039E01D4B0022CB
:101DE0005A8081221A7033E043882BB1194B0022AC
:101DF0005A8082221A702BE01B4B9847012805D08D
:101E0000144B00225A8082221A7021E0114B0022CA
:101E10005A8081221A701BE043882BB10D4B00229F
:101E20005A8082221A7013E0104B984728B9094B48
:101E300000225A8081221A700AE0064B00225A8042
:101E400082221A7004E0034B00225A8082221A7008
:101E500002B070BD7C11002059804000DD114000AF
:101E6000391B40006D1B4000B11B40002D18400085
:101E7000004870477C110020F0B583B0EFF3108369
:101E8000B3FA83F35B09019372B6BFF35F8F00224D
:101E9000364B1A70019E364B1B68364A15682B4428
:101EA0007F2B2AD8324B1C682246334933482844BA
:101EB000334B98472C442F4B1C6000222C4B1A604C
:101EC0002EB10122294B1A70BFF35F8F62B62D4AE3
:101ED000284B196829482C4B98470146D0B1274B0D
:101EE000C31A284842881A44951D4478012C15D0FD
:101EF00044BB802B1CD900242AE01D4A13681468B7
:101F00002C441B1B03F18004204A137843F0010387
:101F10001370C9E70024174B1C6019E01748154FD0
:101F20003E68761B32464119194B98473E600FE0D8
:101F3000104D2C68E41A22461048154B98472C6027
:101F4000002405E00633802B05D90024094B1C60D2
:101F5000204603B0F0BD0948064D2C68E41A22461D
:101F6000C1180B4B98472C600024F1E7FA010020C0
:101F7000C4140020D41400201C150020C413002019
:101F8000D1944000D8140020111C4000D01400202F
:101F90000596400010B5184B9847184B18600DE097
:101FA000174B195D1748184B98470134E4B2174B8B
:101FB0001B689C42F4D30022144B1A604FF0FF318F
:101FC0000120134B9847134B98470128F6D112482C
:101FD000124B9847124B9847024680210848114BF4
:101FE00098470128EAD10E4B984743880633074AA1
:101FF00013600024DBE700BFED764000C81400202A
:10200000441400200082014093634000CC1400205F
:1020100005794000791E4000D8140020E91C4000DA
:10202000711E4000A11C400030B583B080242246C0
:1020300000211B481B4DA847224600211A48A847EB
:1020400000231A4A13601A4A13601A4A13701A4A74
:1020500010215166C2F8901051655162C2F880108B
:10206000116F21F010011167516F21F010015167BC
:10207000124A4FF400211160202182F8131301212C
:102080000F4A91600193009322460E490E480F4C6F
:10209000A047012802D00E480E4B984703B030BD30
:1020A0001C150020CD96400044140020C4140020CC
:1020B000CC140020D0140020000E0E4000E100E0FF
:1020C00000820140A8BF4000951F40009D71400064
:1020D000B0BF40007D8E4000194B1B6913F0010F0B
:1020E0002DD0174B5B6913F0010F28D000B583B0DA
:1020F000144B1B687F2B1CD8124A1368591C1160A3
:102100000F4A9169104AD15402A9002341F8043DB5
:102110000E4B18680E4B9847019B3BB14FF0805215
:102120000C4B1A60BFF34F8FBFF36F8F03B05DF896
:1021300004FB094A137843F001031370E4E7704786
:1021400000820140C41400201C150020C814002087
:10215000717A400004ED00E0D0140020154B984245
:102160001BD003F5A033984219D003F58043984261
:1021700017D0A3F54043984215D003F58043984209
:1021800013D0A3F5A033984211D003F560339842E1
:1021900001D0322070471620704708207047092070
:1021A00070470E2070471320704714207047152089
:1021B000704700BF00C000404900B0FBF1F0033899
:1021C000002302E040080133DBB2FF28FAD8020204
:1021D00002F47F4252FA80F01B0403F4E023184417
:1021E000704700002DE9F843D0F80090037ADBB285
:1021F000012B00F09E80044609F5C065087908B9F6
:10220000BDE8F88317460E46012323720023E371CD
:10221000E1604C4B98478046B378022B08D0737826
:10222000012B18D033781B0403F4FE036B603DE0F0
:102230007378012B09D033781B0403F4FE0303F5F4
:1022400080736B60F378EB6030E033785B081B04DD
:1022500003F58073F5E733785B081B04E6E7032397
:10226000A37100232372237A002B65D02B6A13F409
:10227000807F3BD113F0040F3CD1324B984708EBE1
:1022800007039842F2D90523A371002323722E4B32
:10229000C9F800362EE00423A37100232372E2E77D
:1022A000284B984708EB0703984217D83379E2790F
:1022B0009B1A002BD7DD2B6A13F4807FCFD113F448
:1022C000007FE8D113F0040FEAD0B168E379DBB204
:1022D0005A1CD2B2E271CB5C6B63E1E70523A371B8
:1022E00000232372184BC9F80036BCE70323A371FF
:1022F00000232372237A13B30223C9F800362B6A12
:1023000013F0010F0ED10F4B984708EB07039842CB
:10231000F5D90523A371002020720B4BC9F80036B4
:10232000BDE8F883002323720223A3710120BDE8D6
:10233000F8830020BDE8F8830020BDE8F883002082
:102340005EE700BF35284000028000052DE9F84F08
:10235000D0F800A0037ADBB2012B00F09E800AF5D2
:10236000C0660B7913B91846BDE8F88F17460D46BD
:102370000446012303720023C371E160494B98476F
:102380008046AB78032B14D06B78012B24D02B78AC
:102390001B0403F4FE0303F58053736095F8049067
:1023A000B9F1010F1ED00123CAF800364FF0000921
:1023B0004DE06B78012B09D02B781B0403F4FE034E
:1023C00003F588537360EB78F360E7E72B785B08DD
:1023D0001B0403F58853F5E72B785B081B0403F512
:1023E0008053DAE70323CAF8003630E00323A371F1
:1023F00000232372237A002B51D0336A13F0010F8C
:1024000045D1284B984708EB07039842F5D9052397
:10241000A37100232372244ACAF80026A3E70423E9
:10242000A37100232372E5E70523A3710023237220
:102430001D4BCAF80036DDE71BF0020F07D0A96874
:10244000E379DBB25A1CD2B2E271326BCA54E3793F
:10245000DBB22A799342CDD2D6F820B01BF4807F2C
:10246000C4D11BF4007FDAD10E4B984708EB070369
:102470009842D9D8B9F1000FDED12B79E2799B1AB5
:10248000012BD9D1022333604FF00109D4E7002397
:1024900023720223A371012365E7002363E700236E
:1024A00061E700BF35284000028000052DE9F041BA
:1024B00006468846046820461B4B9847312801D9B8
:1024C000BDE8F0810546194B984703232360242378
:1024D000C4F8003641461648164B9847C4F8100613
:1024E000002333720123B3716BB2002B07DB5A094F
:1024F00005F01F00012181400F4840F82210002BF9
:102500000BDB03F1604303F56143202283F80023D2
:1025100001200A4B98473061D2E705F00F05084BC0
:1025200020225A55F4E700BF5D214000A961400018
:102530000000DC05B921400000E100E0256D40000D
:1025400014ED00E008B54FF0FF310069014B9847EA
:10255000C0B208BD456D400010B500231A461946AB
:102560000069024CA047C0B210BD00BFED6B400037
:1025700008B5837963B18B78032B0BD8DFE803F0C0
:1025800002050205044B984708BD044B984708BD57
:10259000002008BD002008BDE52140004D2340007B
:1025A000F8B50646036803F5C064256AC76815F0E8
:1025B000040F0BD0E26A12F0040F07D0BA78002A99
:1025C0004DD0022A4BD0BA78032A5ED015F0020F04
:1025D00008D0E26A12F0020F04D0BA78012A73D050
:1025E000032A71D015F4807F0DD0E36A13F4807F45
:1025F00009D040F20733A362002333720323B3717F
:10260000FB6803B1984715F4007F0DD0E36A13F41B
:10261000007F09D040F20733A36200233372042302
:10262000B371FB6803B1984715F0010F16D0E36A48
:1026300013F0010F12D0BB780BB1022B09D140F27D
:102640000533A362002333720223B371FB6803B125
:102650009847BB78012B54D0032B52D0F8BDF279A8
:10266000D2B239798A4208D2B868F279D2B2511C12
:10267000C9B2F171825C6263A5E70222C3F8002649
:10268000012262620422A2629DE77A78012A11D0B7
:102690003A78120402F4FE0202F5805262603A793E
:1026A000012A0DD00122C3F800260422A2620222D0
:1026B00062628BE73A785208120402F58052EDE725
:1026C0000322C3F80026F0E7B868F279D2B2511CB1
:1026D000C9B2F171216B8154F179C9B23A79013AE9
:1026E00091420AD0F379DBB23A7993427FF47AAF20
:1026F000012363620223A36274E70222C3F8002667
:10270000F0E740F20333A362002333720223B37174
:10271000FB68002BA2D09847A0E7000070B40568C2
:1027200005F5C0660379202B0BD9A3F12001CBB2AC
:102730001A4C012199402160216521612163002209
:1027400011E0174CF5E701339BB2B3F52F7FFAD3B5
:102750006163002301E001339BB2B3F52F7FFAD30D
:1027600021630132D2B2092A01D80023EDE7616169
:10277000616032698023C5F80036002301E001332F
:102780009BB2B3F52F7FFAD332612423C5F800360C
:10279000002303720123837170BC704700100E4048
:1027A000000E0E40F8B5084C4FF4804666630A20D0
:1027B000064DA847402767630A20A84727630A20D9
:1027C000A8472663F8BD00BF000E0E4055744000B8
:1027D000F8B578B9114D4FF480736B630220104C3B
:1027E000A0474FF080736B630420A04701220D4B7C
:1027F0005A63F8BD094E4FF480737363094F022585
:102800003D632846064CA04701233B630420A047B4
:102810004FF0807333632846A047F8BD000E0E408A
:102820005574400000100E400322014B1A6070479F
:1028300030140E40044B986801E0034B9868024B3B
:102840009B689842F9D1704730140E40014B1880B4
:10285000704700BF9C15002008B5154B1B8807EE7C
:10286000903AF8EE677A9FED137A67EE876AB7EED3
:10287000007A37EE667A9FED106AC6EE276A66EE3A
:10288000877A17EE900A0D4B9847DFED0D7A07EE29
:10289000100A27EE277ADFED0B7A77EEC77ADFEDA5
:1028A0000A6A86EEA77A094B83ED007A08BD00BF5D
:1028B0009C15002001088039FFEF7F45BD80400056
:1028C0003313954300F05745C47D7B49A015002084
:1028D000BFF35F8F024B1868BFF35F8F704700BF75
:1028E000A01500208388B3F59F5F04D0B3F5706F07
:1028F0000ED000207047C288B2F51F6FF6D1428912
:10290000A2F5E752093A92B2C62AEFD801207047E1
:10291000C388B3F5F06F01D0002070474389A3F559
:102920000B53053B9BB2C62B01D8022070470020F9
:102930007047000008B5044B98476420034B984744
:10294000034B9847F7E700BF3D0240005574400035
:10295000592840002DE9F041944B9847944B18605A
:10296000944B9847944B98470222944B1A63944B8C
:1029700098470546002407E00520924B9847904B66
:10298000984705460134E4B20DB9132CF4D98E4BA7
:10299000984729468D4B98478D4B984740F2131026
:1029A000884B98478B4B9847002416E0A2008A4931
:1029B00011F82430501C085C03EB0023901C085CC9
:1029C00003EB00430332895C04F5406003EB0161D3
:1029D0008000824B98470134A4B23F2CE6D90120F5
:1029E0007F4B98471920774B98474FF48072734B71
:1029F0001A637C4B98476F4B98477B4B98477B4BB0
:102A0000984705467A4B9847044678B901246B4BA2
:102A1000DB6B13F4004F16D0764B98470F20764BA4
:102A2000984701466548754B984726E105F194069D
:102A3000604B98473146724B984795F89830002B79
:102A4000E5D00024E3E76F4B9847E7E700206E4DA1
:102A5000A8476E4B18700120A8476D4B187016E1FF
:102A60006C4B984720B16C4B9847002840F014817C
:102A700000226A4B1A70514D4FF480766E63192014
:102A8000504B98472E6307E1634B9847002800F0AE
:102A90000881624B1B78002B40F006810020604EBD
:102AA000B047604D28700120B0475F4B18702B78FD
:102AB000002B00F0F980002800F0F6800127574B2A
:102AC0001F705A4D28465A4B98472846594B9847ED
:102AD00080464FF4FA703B4B98470020B047514D69
:102AE00028703846B047504B18702B7803B118B98E
:102AF00000224A4B1A70D7E0414600204E4DA847AD
:102B000041463846A8474D4D002128464C4B984732
:102B10002B78112B15D0002108464A4DA8470021DB
:102B20000120A8473CB3484B984720B3474B1B783C
:102B3000CBB101210020464DA84701210846A847F6
:102B4000B2E06B78002BE6D1AB78002BE3D1EB78C9
:102B5000892BE0D12E46294600203E4DA84731461C
:102B60003846A847D7E700210846394DA847002135
:102B70000120A84798E001210020354DA8470121F8
:102B80000846A84790E00021334B19702B482C4B86
:102B900098478EE00020314B1870214DA847214BFB
:102BA00018700120A847204B187087E0ED76400090
:102BB000F40B00205980400065134000000E0E40C9
:102BC0009D0240005574400051804000DD144000DB
:102BD000A527400091174000D0BF4000FD174000DE
:102BE000D1274000010E400081124000051B40002B
:102BF000D91B4000B50A4000875D4000635D40007E
:102C0000DD114000910A4000410D4000B10000205C
:102C1000B2000020A5804000B1804000E80B0020F9
:102C2000F1184000E60B0020E70B00207C16002086
:102C30002D194000E5284000990D40002416002081
:102C400049184000D90C4000850E4000B300002018
:102C5000FD0C4000850D4000E40B0020E50B00203A
:102C60002C4B984730B101222B4B1A702B4B1B7801
:102C7000002B41D10A202A4B9847284B1B78002B68
:102C80007FF4E4AE4723274A1370274A1370234B7F
:102C90001B78002B7FF4E4AE244B984700287FF488
:102CA000F3AE00221D4B1A70214B1B78002B7FF4D2
:102CB0006AAF204B1B78002B7FF46CAF1E4B9847FC
:102CC00010B31E4B9847002CD4D0134B1B78002B0D
:102CD000C6D0104B98470028CCD100220E4B1A705A
:102CE0000E4B1B78002BC5D011461046144DA8473B
:102CF00000210120A847BDE711460020104DA8473C
:102D000001210846A847B5E70E4B98476420044BBD
:102D10009847B2E7E50E4000B3000020E80B002022
:102D200055744000B1000020B2000020A580400092
:102D3000E40B0020E50B0020850E4000910E4000C2
:102D4000FD0C4000010E400008B5284B9847284B69
:102D5000186006E000210846264CA047002101200B
:102D6000A0474FF0FF310120234B9847234B1B789E
:102D7000013B062BF5D801A252F823F0992D400013
:102D8000552D4000BB2D4000CB2D4000A92D40000B
:102D9000DB2D4000E72D400001210020154CA0470D
:102DA00001210846A047DCE7154D29880020154C75
:102DB000A04729880120A047D3E700210846124CEC
:102DC000A04700210120A047CBE7012100200E4CA5
:102DD000A04701210846A047C3E70C4B98470C4980
:102DE0000C4B9847BDE70C4B9847BAE7ED7640008F
:102DF000EC0B0020210D400005794000A7150020B4
:102E000088160020890C4000FD0C400059804000CD
:102E1000A4150020DD114000B11B4000F8B5524B55
:102E20009847524B18604FF47A72514B1A804022E7
:102E300000215048504B984734E0504B98474D4A3A
:102E400055231370202353704D4B1B7800EB431018
:102E5000076846688568C168C2F80270C2F80660F3
:102E6000C2F80A50C2F80E10076946698569C1693F
:102E7000C2F81270C2F81660C2F81A50C2F81E10DA
:102E80001AE03C484D2303703E4B1A7842701A7882
:102E90003D4902303D4B984710E040220021354823
:102EA000354B9847324B198889B20120384B9847E7
:102EB000044658B15528C0D04D2CE2D0354B984728
:102EC0000028EAD02B48344B9847E6E7294C2323C7
:102ED000237014236370314B9847C0F30F23A37002
:102EE000E0702F4B9847C0F30F23237160712D4B77
:102EF0009847C0F30F23A371E0712B4B9847C0F3A1
:102F00000F2323726072294B9847C4F80A00284B9C
:102F10001B7807EE103AB8EE477A9FED266A27EE47
:102F2000067ADFED256A37EE667A17EE103AC4F8B6
:102F30000E30224B1B7807EE903AF8EE677A67EE78
:102F4000867A77EEE67A17EE903AC4F81230114B93
:102F5000984728B9402200210648074B9847A1E727
:102F600020460D4B9847F5E7ED764000F00B00202A
:102F700022160020CC150020CD964000391B4000C1
:102F800020160020211600208C160020D19440002D
:102F9000057940007980400089334000250A4000CF
:102FA000F10E40008502400091024000D12840000F
:102FB000B1000020B4C8363F6FDB4A42B2000020A7
:102FC00010B582B00023019301220092802219499A
:102FD00019481A4CA047012802D01948194B9847A4
:102FE0000023019303220092802217491748134CB3
:102FF000A047012802D01648124B9847002301939E
:1030000000938022134914480C4CA047012802D099
:1030100012480C4B984700230193009380221049DB
:103020001048064CA047012802D00F48054B98478E
:1030300002B010BDD0C040001D2E40009D71400068
:10304000D8C040007D8E4000FCC04000492D4000AB
:1030500000C140001CC140005529400028C140006B
:1030600050C140003529400054C1400030B585B002
:1030700004460378532B25D02378472B2CD0237874
:10308000672B37D02378462B3CD02378522B3DD06A
:103090002378502B44D02378492B64D02378422BBB
:1030A0007ED0552B00F08E802378572B00F0A8801F
:1030B0002378562B00F0AE8023784C2B00F0C28092
:1030C00005B030BD43781BB901206E4B9847D3E75C
:1030D00000206C4B9847CFE76378A07800EB032083
:1030E00080B210F4004F02D1674B9847C7E747F60C
:1030F000FF70F9E76378A07800EB032000B2634B20
:103100009847BFE76078624B9847BEE76278A3783C
:1031100003EB02239BB2092BBAD95E4A1380B7E7AF
:103120006378B3B902225C4B1A7004A9002341F8FA
:10313000043D5A4B18685A4B9847039B002BAAD062
:103140004FF08052574B1A60BFF34F8FBFF36F8F12
:10315000A1E7012B03D000224F4B1A70E5E70122B3
:103160004D4B1A70E1E76278A37803EB02234E4AD5
:1031700013800522484B1A7004A9002341F8043D2E
:10318000464B1868464B9847039B002B86D04FF060
:103190008052444B1A60BFF34F8FBFF36F8F7DE7B0
:1031A000424BBB221A601A225A60BFF34F8F40492C
:1031B000CA6802F4E0623F4B1343CB60BFF34F8F0A
:1031C00000BFFDE763780F2B3FF66EAF3A4A1370EE
:1031D000002304AA42F8043D3849086800920322FB
:1031E0005521374DA847039B002B3FF45DAF4FF0AF
:1031F00080522C4B1A60BFF34F8FBFF36F8F53E792
:1032000061780F293FF654AF20224901A01C2D4BB5
:1032100098474DE70722204B1A7004A9002341F874
:10322000043D1E4B18681E4B9847039B002B3FF430
:1032300043AF4FF080521B4B1A60BFF34F8FBFF369
:103240006F8F39E7204B62781A70A2785A70E27853
:103250009A700622104B1A7004A9002341F8043D0D
:103260000E4B18680E4B9847039B002B3FF428AF7A
:103270004FF080520B4B1A60BFF34F8FBFF36F8F2D
:103280001EE700BF89364000513640007D364000C1
:10329000D909400022160020A7150020EC0B0020C1
:1032A000717A400004ED00E08816002090140E4072
:1032B00000ED00E00400FA0520160020F00B0020CD
:1032C000897940006D1B4000A41500200023044AAA
:1032D0001370044A13700120034B1870704700BF2D
:1032E000000C0020FC0B0020F80B00207047002091
:1032F000704700000D4B5B881A0A032A01D000209A
:10330000704713F0FF0F0ED1084BDB88402B01D024
:1033100000207047054B064A9A60064A1A6140220F
:103320009A81012070470020704700BF381B0020A1
:10333000040C0020693340000122014B1A707047D1
:10334000F80B002010B5034B034A04490448054C10
:10335000A04710BDF532400084010020FC0B002086
:10336000000C00208934400008B5044B9B89402B99
:1033700000D008BD0248034B9847FAE7381B0020ED
:10338000040C00206D304000224B1B780BB918460E
:1033900070472DE9F04184B00746EFF31083B3FA8C
:1033A00083F35B09039372B6BFF35F8F00211A4B5F
:1033B0001970DDF80C80194D40222846184B9847AB
:1033C0003C4640372E4620686168A268E3680FC615
:1033D00010343546BC42F5D1124B009340230F4ABE
:1033E00000218120104CA04780F00100094B18708B
:1033F000B8F1000F05D00122074B1A70BFF35F8FA1
:1034000062B6044B1B7883F00103184604B0BDE894
:10341000F08100BFF80B0020FA010020440C0020CE
:10342000CD964000393340007958400010B504462D
:10343000134B9847837A212B01D0002010BD00F157
:103440000902104B5B881B0A212B04D0C27B9342DC
:103450000BD0002010BD0B4B9A60427AD9888A426B
:1034600028BF0A469A81012010BD064B9C60028A43
:10347000D9888A4228BF0A469A81012010BD00BF20
:10348000253D4000381B0020F8B5264C247865B255
:10349000002D07DB002D40DB04F06004202C22D03F
:1034A0000020F8BD14F0600603D11E4F7F78062F70
:1034B0000BD0202EEED11B4A5278022A09D0032AC3
:1034C0000CD0012AE6D19847F8BD1046164B984714
:1034D000F8BD144B986001209881F8BD114B99609C
:1034E00001209881F8BD0F4A52780A2A07D00B2A8A
:1034F0000BD0092A01D00020F8BD9847F8BD094B30
:103500005B881B0A03700120F8BD064BDB8833B9CA
:10351000044B5B880B700120F8BD0020F8BD002033
:10352000F8BD00BF381B00202D34400070B590B0AE
:1035300000248DF835408DF836408DF837408DF8F1
:1035400039408DF83A40ADF83E400F238DF83430C5
:103550000A23ADF83C3001258DF838500DAA0B49EF
:1035600007A80B4EB0470DAA0A4901A8B04710237F
:10357000079A1360019A1360074B1D70074B1C706C
:1035800047F6FF72064B1A8010B070BD00C00240B3
:10359000915C400000000340840C00208C18002047
:1035A0005619002042B110B420B119B1034B586034
:1035B00099605A805DF8044B704700BF840C00206E
:1035C000154B1B783BB3144B5B8823B3124A5268EC
:1035D0000AB311498968F1B1F0B583B00092019343
:1035E0000E4D6A46694628460D4FB8474FF480365F
:1035F0002E62094B9B6800930A4C6A466946204636
:10360000B847266201212846074DA84701212046D8
:10361000A84703B0F0BD7047840C002000C10240F1
:10362000CD5B400000010340E55B4000064B1B788A
:103630003BB1054B5888054BD3F80431C01A80B212
:1036400070470020704700BF840C002000C002407B
:10365000094AD36D23F4FF4323F07F03C0F30E0028
:103660000343D36502F58042D36D23F4FF4323F077
:103670007F031843D065704700C00240014B18809B
:10368000704700BF56190020014B1870704700BFEB
:103690008C180020004870475819002000487047D7
:1036A000AC160020704770472DE9F8434C4B984703
:1036B00005464C4B9847044678E0A0EB070E1FFAEE
:1036C0008EFE0EF1F00E1FFA8EFE7EE031210023F9
:1036D00008E02F21FBE744480078C0B2012831D030
:1036E00001339BB2994252D9DA1992B2EF2A01D929
:1036F000F03A92B23C4800780028ECD13B48B0F94F
:10370000000035F9126006FB00F6F6134FEA830855
:10371000DFF8E0C00CF8236008F10109C6F30726C2
:103720000CF8096034F9122000FB02F2D21308F100
:1037300002000CF8002008F10308C2F307220CF87D
:103740000820CDE735F9120034F91220024402EBCB
:10375000D272521012F5004F05DBB2F5004F03DBB9
:1037600047F6FF7200E0224A98005FFA82FC214E81
:1037700006F823C000F10108C2F3072206F808206A
:1037800000F1020806F808C003303254A8E71A4BCB
:10379000A3F800E07744BFB2184B1F80EF2F01D988
:1037A000F03F1F8089001348154B98474FF0FF31B9
:1037B0000120144B9847144B9847104B1F88B84270
:1037C000FFF47BAFC01B1FFA80FEBEF1300F3FF647
:1037D0007DAFBEF12F0F7FF67CAF302177E700BFC2
:1037E000953640009D3640008C1800205619002068
:1037F0000080FFFF9018002054190020900C00203A
:1038000099034000057940002D364000024B1B68AB
:103810001B68588818447047A00C002038B504462F
:103820000D46094B9847024620782044904207D223
:103830004378042B06D0AB4205D003781844F5E753
:10384000002038BD002038BD0D38400038B5144B7D
:103850001B780BB3134B1B681B681A7982421DD966
:103860000D460446104A1360104B984703E01A783F
:1038700013440D4A13600C4B1B6898420AD95A78BE
:10388000042AF4D19A789442F1D1DA78AA42EED19E
:10389000012038BD002038BD002038BD002038BDD3
:1038A0009C0C0020A00C0020A40C00200D3840002F
:1038B000084BDB8863B9074B5B88012B01D00020E4
:1038C0007047054A138823F00203138001207047D4
:1038D00000207047381B0020920C00200020704709
:1038E000044BDB8823B9044A024B1A61012070475C
:1038F00000207047381B0020153C400038B5134BA2
:103900001B7803B3124B1C79124B1B681B681B7985
:103910009C4201D3002317E0002120460E4B98471C
:10392000034688B10B4B1B685B6853F82450EB6867
:10393000984701462046084B9847034620B1AB689C
:103940009847034600E00023184638BD9C0C002031
:10395000381B0020A00C00204D38400038B5104B1B
:103960001B78D3B100240F4B1B681A68127994425C
:1039700011D25B6853F82450EB6898470146204603
:10398000094B9847034648B1AB689847034628B9A6
:103990000134E4B2E7E7002300E00023184638BD15
:1039A0009C0C0020A00C00204D38400070B504464F
:1039B0000021114B9847054608B9284670BD0F4BAA
:1039C0001B685B6853F82460F368984701462046FB
:1039D000094B984705460028EFD0094B1C68052184
:1039E0002046084B9847044618B18078064B984704
:1039F000F5E773689847E0E74D384000A00C0020D9
:103A0000A40C00201D384000F955400008B5064BB5
:103A1000DB88022B01D0002008BD02210348044BA3
:103A20009847012008BD00BF381B0020920C0020E1
:103A3000DD54400010B5154B9B78012B04D043B1E9
:103A4000022B0CD0002010BD0720114C50B10023D8
:103A500011E004210F48104B98470020F6E715208D
:103A60000E4CF3E7012010BDE15C0D4A02EB43026E
:103A700051800133DBB28342F6D3411C4900C9B205
:103A800007480170044B9847012010BD381B0020E7
:103A9000DC010020D8010020DD544000E4010020BA
:103AA000AC01002008B5234B5B88DAB21B0A013B4E
:103AB0000E2B38D8DFE803F00817313737373737A0
:103AC0003737373737372A001B4B186801781B4BBD
:103AD0009847184BDA889B899A4228D2154B9A81CD
:103AE0000123184608BD144B1B685B7C9A4201D326
:103AF0000023F6E7104B5B6853F8320041880F4B08
:103B000098470C4B9B6802225A70E2E70A4B986870
:103B100058B14188094B9847DBE7094B9847034662
:103B20000028D6D1DDE70023DBE70023D9E7012316
:103B3000D7E700BF381B0020B4000020DD54400050
:103B4000353A400008B5064BDB88012B01D0002038
:103B500008BD01210348044B9847012008BD00BF60
:103B6000381B00209C0C0020DD54400038B5154B5C
:103B7000DB88012B02D00024204638BD124B1B7875
:103B8000F3B1104B1D79114B1B681B681B799D42CB
:103B900001D30024F0E7002128460D4B9847044646
:103BA0000028E9D0094B1B685B6853F82530DB68B7
:103BB0009847084B187001211846074B9847DBE7D8
:103BC0000024D9E7381B00209C0C0020A00C00200A
:103BD0004D384000980C0020DD54400008B5094BDA
:103BE000DB88022B01D0002008BD064B1879064B5C
:103BF0009847064B188002211846054B984701202C
:103C000008BD00BF381B002049564000940C00201E
:103C1000DD54400008B5034B588800F07F00024B8C
:103C2000984708BD381B00208554400038B505462C
:103C30000F4B98470346C0B10E4B1C680521204628
:103C40000D4B9847044640B18288C17880780B4B71
:103C5000984703460028F1D107E0094B1B685B68D1
:103C600053F825301B6898470346184638BD00BFF7
:103C70004D384000A40C00201D384000E95440009D
:103C8000A00C002038B50C4BDB8893B90B4B1B788C
:103C90000BB900230EE0084B1C799D782046084B99
:103CA0009847034630B129462046064B98470346BD
:103CB00000E00023184638BD381B00209C0C002073
:103CC000AD3940002D3C400008B5074BDB884BB9AF
:103CD000054B5B880BB1002008BD034B1879034BE3
:103CE000984708BD002008BD381B002085574000BC
:103CF000094BDB886BB9084B5B880BB10020704720
:103D000010B5054C2079054B98472079044B98470E
:103D100010BD0020704700BF381B0020F55940003F
:103D20008D564000014B1868704700BFA40C00205E
:103D300008B5014B984708BDC153400010B50B4B67
:103D40001B7863B1002404E02046094B98470134F6
:103D5000E4B2084B1B681B681B799C42F4D3002219
:103D6000024B1A700122044B1A8010BD9C0C0020DB
:103D7000AD394000A00C0020920C00201C4BDB88C9
:103D800013B100231846704710B51A4B984750B32B
:103D9000174B9A78184B1B685B7C9A4201DD002315
:103DA00022E0164B9847124B9B78154A1370EBB1E3
:103DB000114A526803F10053013B02EBC303114A5D
:103DC000136000240F4B1B681B681B799C4208D2B0
:103DD000002120460C4B9847034628B10134E4B239
:103DE000F0E7012300E00023184610BD0123FBE7A4
:103DF000381B0020C1544000B40000203D3D40006D
:103E00009C0C0020A00C00202D3C400008B5344B39
:103E10001B7813F0800F0ED113F01F0343D1304AEB
:103E20005278013A082A3ED8DFE802F0343D373DA7
:103E3000313D3D3D3A002A4AD288002A4ED013F047
:103E40001F0306D1264A5278062A0BD0082A0CD026
:103E50002AB1012B0CD0022B11D0002008BD214B20
:103E6000984708BD204B984708BD204B984708BD90
:103E70001B4A52780A2AEED11D4B984708BD184BB1
:103E80005B780BB1002008BD1A4B984708BD1A4B50
:103E9000984708BD194B984708BD194B984708BD6E
:103EA000184B984708BD012B03D0022B08D00020E7
:103EB00008BD0B4A52780B2AF7D1134B984708BD1F
:103EC000074B5B78012B03D0032B04D0002008BDE7
:103ED0000E4B984708BD0E4B984708BD002008BD03
:103EE000381B00200D3A4000A53A4000453B4000F9
:103EF0006D3B4000DD3B4000E1384000B138400000
:103F0000DD3840007D3D4000853C4000C93C40001C
:103F1000F13C40000B4B1B7813B110B5002402E0BC
:103F200070470134E4B2084B1B681A681279944256
:103F300007D25B6853F824301B69002BF1D09847F7
:103F4000EFE710BD9C0C0020A00C002008B5184B1A
:103F500000229A811A615A611B7813F0800F11D1E7
:103F600013F0600F14D0124B1B7803F01F03012BCA
:103F700014D00F4B1B7803F01F03022B14D0002327
:103F8000184608BD0A4AD288002AE9D10023F7E77B
:103F9000084B984703460028E5D0F1E7064B9847C1
:103FA00003460028E5D0EBE7044B98470346E7E7D4
:103FB000381B00200D3E4000FD3840005D394000B8
:103FC000F8B504460E46114B984705462046104B5F
:103FD0009847054001D0002403E0F8BD0134062CC9
:103FE00011D88DB123010B4AD058B042F6D102EB63
:103FF000041359680D42F1D01F46DB6898477B686F
:1040000025EA0305EAE7F8BDF8BD00BF6B5D400097
:104010006F5D4000A80C0020F8B5164C2768062FED
:1040200026D8002401E00134E4B2A446A7420AD312
:10403000114E250106EB050E75598D42F3D1DEF8C0
:1040400004509542EFD1CEF80010CEF80420CEF8FF
:1040500008300699CEF80C100137BC4505D0114642
:104060001A46064B98470020F8BD02490F60F6E754
:104070000120F8BD180D0020A80C0020315D400083
:104080002DE9F04182B004460F4690460A4B98470E
:1040900005462046094B984706462046084B984758
:1040A000CDF800803B46024631462846054CA047E5
:1040B00002B0BDE8F08100BF735D4000815D40004B
:1040C000875D40001940400008B50B210148024BB4
:1040D000984708BD000E0E40C13F400008B50C21B6
:1040E0000148024B984708BD00100E40C13F4000F8
:1040F000F8B506460C461546224B984707464FF042
:10410000FF313046204B98473046204B9847002CD3
:104110000CDB630904F01F0101228A4020331C4993
:1041200041F82320BFF34F8FBFF36F8F002C08DBC4
:10413000630904F01F0101228A406033144941F8E9
:104140002320002C17DB2D01EDB204F1604303F5B1
:10415000614383F80053002C08DB620904F01F045C
:10416000012303FA04F40A4B43F82240394630464F
:10417000084B9847F8BD04F00F022D01EDB2064B35
:104180009D54E8E76F5D4000675D40006B5D400057
:1041900000E100E0635D400014ED00E082B0024603
:1041A00010B9244B1B783BB912B1224B1B780BB3CF
:1041B000204B1A7002B070471F4B1B7803B9FEE703
:1041C000EFF31083B3FA83F35B09009372B6BFF386
:1041D0005F8F0021194B1970009817490B78013B2C
:1041E0000B700028E0D00121144B1970BFF35F8FD2
:1041F00062B6D9E7104B1B78FF2B19D0EFF3108371
:10420000B3FA83F35B09019372B6BFF35F8F0021AA
:104210000A4B1970019808490B7801330B7000287C
:10422000C6D00121054B1970BFF35F8F62B6BFE79F
:10423000FEE700BF1D0D0020501B0020FA010020EA
:1042400084B02A4B9A6842F480729A609A6822F08D
:104250007F029A601A6B0192019A42F04F0201921A
:10426000019A22F4074222F080020192019A42F45C
:1042700000420192019A1A631C4B1B6B13F4004F0E
:10428000FAD01A4A136B0293029B43F04F03029336
:10429000029B43F400430293029B136300238DF8B7
:1042A000033006E000BF9DF803300133DBB28DF828
:1042B00003309DF80330DBB2132BF3D9EFF31083F7
:1042C000B3FA83F35B09039372B6BFF35F8F0022E7
:1042D000074B1A70039B0121044A116123B1044B5F
:1042E0001970BFF35F8F62B604B07047004004409E
:1042F000FA010020034A0023136153619381024AAB
:1043000013707047381B0020220D002082B0052258
:10431000104B1A70104A136B0193019B43F04F032B
:104320000193019B43F020030193019B136300233E
:104330008DF8033006E000BF9DF803300133DBB297
:104340008DF803309DF80330DBB2132BF3D902B0A4
:10435000704700BF220D00200040044082B00322BD
:10436000104B1A70104A136B0193019B43F04F03DB
:104370000193019B43F010030193019B13630023FE
:104380008DF8033006E000BF9DF803300133DBB247
:104390008DF803309DF80330DBB2132BF3D902B054
:1043A000704700BF220D0020004004400422014B52
:1043B0001A707047220D002008B5024B1B6903B12B
:1043C000984708BD381B002030B589B06A4B1B7870
:1043D000032B29D0694B9C89694B1B88E41AA4B232
:1043E000002C43D1674A11880B449BB21380634A67
:1043F000D288934203D0644B1B78002B2CD0634BA4
:104400009847634A136B0393039B43F04F03039353
:10441000039B23F001030393039B13635C4B1B6B10
:1044200013F0010FFAD115E0594A136B0293029B66
:1044300043F04F030293029B23F001030293029B7C
:104440001363534B1B6B13F0010FFAD1514B984779
:10445000514B984709B030BD484B5B6933B1984721
:1044600020B10022464B1A80444B9C893F2C37D9FF
:104470000022454B1A704024404B9A68404B1B88E1
:104480001A44EFF31083B3FA83F35B09079372B610
:10449000BFF35F8F0021414B197007983C4B1B6B9A
:1044A00013F0020F3ED028B101223C4B1A70BFF32B
:1044B0005F8F62B60422304B1A70354A136B049337
:1044C000049B43F04F030493049B23F001030493E4
:1044D000049B13632E4B1B6B13F0010FFAD1B9E74A
:1044E0000122294B1A70C7E7157829490D65013358
:1044F000DBB2013299B28C42F6D8214B1A881444AF
:104500001C80234A136B0593059B43F04F030593CF
:10451000059B43F010030593059B136300238DF85F
:10452000073008E00023E5E700BF9DF807300133BE
:10453000DBB28DF807309DF80730DBB2132BF3D9CF
:10454000134A136B0693069B43F04F030693069B97
:1045500023F001030693069B13630D4B1B6B13F0B3
:10456000010FFAD100283FF475AF01220B4B1A70EE
:10457000BFF35F8F62B66DE7220D0020381B00206D
:104580001E0D0020200D00201C0D0020AD4340001A
:1045900000400440B9434000F5424000FA010020C9
:1045A00010B586B0654B1B78012B1ED0022B04D0B2
:1045B000042B02D0624B984701E0624B9847624A55
:1045C000136B0093009B43F04F030093009B23F079
:1045D00002030093009B13635B4B1B6B13F0020FF2
:1045E000FAD15A4B984706B010BD574B186BC0F321
:1045F0000A40574B9B89574A14882218934201DA84
:10460000181B80B2524B9A682244002305E04E49A1
:10461000096D11700133DBB2013299B28842F6D8CC
:104620000444A4B24B4B1C8040281BD0484B9C81B7
:104630005B6913B19847002832D0434A136B029349
:10464000029B43F04F030293029B23F00203029369
:10465000029B13633C4B1B6B13F0020FFAD13E4BD2
:104660009847C0E73A4BDA883C4B1B8823449A4270
:10467000DCDD374B9B899C4227D0334A136B059373
:10468000059B43F04F030593059B23F0020305931D
:10469000059B13632C4B1B6B13F0020FFAD1A2E79F
:1046A000274B9847284A136B0193019B43F04F0314
:1046B0000193019B23F002030193019B1363224B9F
:1046C0001B6B13F0020FFAD18DE7214B5B6953B1DD
:1046D0009847E8B121491F4A0B88108803440B8092
:1046E00000231380C9E7164B9847174A136B0393AF
:1046F000039B43F04F030393039B23F002030393B5
:10470000039B1363104B1B6B13F0020FFAD16AE784
:104710000B4B98470C4A136B0493049B43F04F03D5
:104720000493049B23F002030493049B1363064B3E
:104730001B6B13F0020FFAD155E700BF220D0020CA
:104740000D434000B943400000400440F5424000A2
:10475000381B00201E0D00205D434000200D00206E
:104760000023042B14D810B40A499A00D418A000CE
:1047700004460844407C214400F083026FF3C712D2
:104780004A740133DBB2042BEED95DF8044B704759
:10479000704700BF240D002038B5437C13F0100F84
:1047A00016D00D46437C6FF30413437404687CB148
:1047B00002F10C03074951F8233013F4806F01D044
:1047C00042F080028168012D14BF00200120A04723
:1047D00038BD00BF0040044010B500240BE0234664
:1047E0000134E4B203EB8303980022460121034B1A
:1047F0001844034B9847042CF1D910BD240D002018
:104800009947400010B500F00F02531E03EB8303DD
:104810009C00012102482044024B984710BD00BF74
:10482000240D00209947400030B482B00246441E57
:104830003B4900F10C0551F8253051F8251013F0D3
:10484000020302D001F0400151B9002B39D004EB32
:1048500084039900334B0B44597C6FF383015974E3
:1048600004EB840399002F4B0B445B7C13F00C0F7B
:1048700032D12B4900F10C0551F825300093009BF3
:1048800043F04F030093009B23F002030093009B2F
:1048900041F8253002F10C03214951F8233013F07F
:1048A000020FF7D1002838D0032836D004EB840457
:1048B000A2001C4B13445A7C012161F383025A74F9
:1048C0002BE004EB84039900164B0B44597C012523
:1048D00065F383015974C3E711490C3051F8203056
:1048E0000193019B43F04F030193019B23F040038D
:1048F0000193019B41F8203002F10C03084951F863
:10490000233013F0400FF7D104EB8404A200054BD1
:1049100013445A7C6FF383025A7402B030BC704760
:1049200000400440240D0020F0B4461EB300334480
:1049300099002A4A0A445368D1680B449468641A5F
:10494000128AC2F30902944209D31446002706EBE7
:1049500086029500214A2A442144D1601EE00127A5
:10496000F5E71D781E4A00F1140142F821505D78E8
:1049700042F821509D7842F82150DD7842F82150CC
:104980001D7942F821505D7942F821509D7942F815
:104990002150DD7942F82150083C0833072CE0D83B
:1049A00007E01D7800F114020D4941F82250013C46
:1049B0000133002CF5D1094BB10088198200104653
:1049C0001A44527CC2F3810203440132597C62F3DF
:1049D000830159743846F0BC704700BF240D002095
:1049E0000040044070B582B0441E04EB84039A007A
:1049F000364B13445B7CC3F3810328B1032801D0F9
:104A0000022202E0012200E001229A4254DDA200CB
:104A1000224495002D4B2B44DA689B689A4205D3BB
:104A20002A4B2B445B7C13F0400F48D00E460546C2
:104A3000274B9847FEB1274A0C3552F82530019391
:104A4000019B43F04F030193019B43F0100301933B
:104A5000019B42F8253000238DF8033006E000BFAB
:104A60009DF803300133DBB28DF803309DF803303D
:104A7000DBB2132BF3D940B104EB84039A00134B40
:104A800013445A7C6FF386125A74A2002244910098
:104A90000E4B0B44DA689B689A4212D30B4B0B44C3
:104AA0005B7C13F0400F0ED1084B0B445A7C42F054
:104AB00080025A74002000E0012002B070BD002086
:104AC000FBE70120F9E70120F7E700BF240D0020F4
:104AD00029494000004004402DE9F843054684463A
:104AE000471EBB003B449A002A4C1444A268E3686A
:104AF000A2EB030EB4F81080C8F3090862681A44E8
:104B00000C30254951F82060C6F30A4666B3B64515
:104B10000BD9B6464FF0000907EB870188001D4905
:104B200001447344CB6000210AE04FF00109F3E730
:104B30000CF11403184850F823301370013101327E
:104B40008E45F5D82846154B9847B9F1000F01D18D
:104B5000B04507D905F10C030F4A52F8233013F082
:104B6000200F04D0BDE8F8834FF00009EAE70123E5
:104B7000AB405361074ABB00D81981000846114475
:104B8000C968024491602A4600212046044B984798
:104B9000E8E700BF240D0020004004402948400001
:104BA000994740002DE9F0418CB00124ADE1204649
:104BB000B34B98470120FAE1BB003B449900B14A4E
:104BC0000A44537CC3F38101033161F383035374BB
:104BD000537C13F0200F00F0848013F00C0F3BD0B7
:104BE000A94A04F10C0152F821300193019B43F0D2
:104BF0004F030193019B43F010030193019B42F883
:104C0000213000238DF8013006E000BF9DF801300F
:104C10000133DBB28DF801309DF80130DBB2132B8C
:104C2000F3D9994A06F10C0152F821300293029B04
:104C300043F04F030293029B23F001030293029B74
:104C400042F8213006F10C038F4A52F8233013F05A
:104C5000010FF7D10120AAE18B4A04F10C0152F8AF
:104C600021300393039B43F04F030393039B23F0F3
:104C700001030393039B42F8213006F10C03824A9F
:104C800052F8233013F0010FF7D1114606F10C034F
:104C900052F823200492049A42F04F020492049A9C
:104CA00042F020020492049A41F8232000238DF858
:104CB000023006E000BF9DF802300133DBB28DF810
:104CC00002309DF80230DBB2132BF3D907EB8707D4
:104CD000BA006C4B13445A7C6FF345125A7401208E
:104CE00065E113F0800F42D1BB003B449A00654B55
:104CF0001344DA689B689A424CD307EB87039A0007
:104D0000604B13445B7C13F04C0F43D1EFF31083E3
:104D1000B3FA83F35B090B9372B6BFF35F8F002284
:104D20005A4B1A700B9B584A55612BB10122574BB5
:104D30001A70BFF35F8F62B6534A06F10C0152F846
:104D400021300593059B43F04F030593059B23F00A
:104D500001030593059B42F8213006F10C034A4AF2
:104D600052F8233013F0010FF7D101201FE1BB00EF
:104D70003B449A00434B1344597C6FF3C711597459
:104D8000DA689A60404B5D61224600214046404B04
:104D90009847A9E7002C4AD0032C48D007EB87039B
:104DA0009A00384B13445B7C13F00C0F3FD0364A0B
:104DB00006F10C0152F821300693069B43F04F0395
:104DC0000693069B43F010030693069B42F821309E
:104DD00000238DF8033006E000BF9DF80330013357
:104DE000DBB28DF803309DF80330DBB2132BF3D91F
:104DF000254A06F10C0152F821300793079B43F036
:104E00004F030793079B23F001030793079B42F887
:104E1000213006F10C031C4A52F8233013F0010F25
:104E2000F7D1002120461B4B98470120BFE0002C02
:104E30004AD0032C48D001212046164B984758B33E
:104E4000114A06F10C0152F821300893089B43F0F7
:104E50004F030893089B23F001030893089B42F833
:104E6000213006F10C03084A52F8233013F0010FE9
:104E7000F7D100212046074B9847012097E000BF5B
:104E8000D94A4000240D002000400440FA010020CF
:104E900099474000E54940004749BB00D8198200C6
:104EA0000A4492F811E06FF3C71E82F811E0D2684D
:104EB0001F44BB0019448A60404B5D6122460021BB
:104EC00040463F4B9847BBE7012120463D4B984762
:104ED0003A4A06F10C0152F821300993099B43F03C
:104EE0004F030993099B23F001030993099B42F89F
:104EF000213006F10C03314A52F8233013F0010F30
:104F0000F7D1012053E00134E4B2052C4ED82B4BED
:104F10009B6926460125A5402B42F4D0671E07EB6E
:104F200087029300244A02EB030804F10C03234A8E
:104F300052F8233013F0420F7FF439AE04F10C0322
:104F40001E4A52F8233013F0010F7FF435AE04F1FE
:104F50000C031A4A52F8233013F0080FD3D004F18F
:104F60000C0152F821300A930A9B43F04F030A9335
:104F70000A9B23F008030A930A9B42F8213006F1AA
:104F80000C030E4A52F8233013F0080FF7D106F144
:104F90000C0352F8233003F4E063B3F5807F09D0AB
:104FA00006F10C0352F82330012000E000200CB081
:104FB000BDE8F0810120FAE7240D00200040044004
:104FC00099474000E549400000B587B0534B1B7836
:104FD000E3B9534B1B6BC3F30A43082B3BD0504A36
:104FE000136B0193019B43F04F030193019B23F04B
:104FF00004030193019B1363494B1B6B13F0040FD4
:10500000FAD1484B984707B05DF804FB464B9847E8
:10501000464B9847DDE7424A116D454A99540133A2
:10502000DBB2072BF7D9434B9847B0B93C4A136B17
:105030000293029B43F04F030293029B23F004036D
:105040000293029B1363364B1B6B13F0040FFAD1D0
:10505000344B9847D7E70023E3E7354B93F900300B
:10506000002B1EDB2E4A136B0593059B43F04F0369
:105070000593059B23F004030593059B1363284BBD
:105080001B6B13F0040FFAD1294BDB88002B42D0A5
:105090000023294A1380294A138001221F4B1A70CA
:1050A000B1E71F4A136B0393039B43F04F03039332
:1050B000039B43F080030393039B136300238DF84A
:1050C000033006E000BF9DF803300133DBB28DF8FA
:1050D00003309DF80330DBB2132BF3D9104A136B66
:1050E0000493049B43F04F030493049B23F00403B5
:1050F0000493049B13630A4B1B6B13F0040FFAD148
:1051000000230D4A13800D4A13800222034B1A70AC
:105110000B4B984777E70B4B984774E7220D00201D
:10512000004004400D434000B9434000F5424000B8
:10513000381B00204D3F4000200D00201E0D002098
:10514000C94340005D434000204BDB6913F0010F71
:1051500037D000B583B01D4B1B6B13F0040F24D167
:105160001A4B1B6B13F0010F23D1184B1B6B13F061
:10517000020F22D1154B1B6B13F0080F23D0134ADB
:10518000136B0193019B43F04F030193019B23F0A9
:1051900008030193019B13630C4B1B6B13F0080F67
:1051A000FAD1012003B05DF804FB094B98470120B8
:1051B000F8E7084B98470120F4E7074B9847012090
:1051C000F0E7002070470020ECE700BF00400440FB
:1051D000C94F4000C9434000A145400010B54C4BA9
:1051E000984720B94B4BDB6913F4807F10D03020F7
:1051F000494B9847474B9B6913F4006F04D0454BCC
:10520000DB6913F4006F0AD1444B984770B110BDAD
:1052100072B6BFF35F8F0022414B1A7010BD4FF47E
:1052200000623C4B1A623F4B984710BD3E4B98477B
:105230000028ECD1374B9B6913F4005F04D0354B49
:10524000DB6913F4005F3DD1324B9B6913F4007F9F
:1052500004D0304BDB6913F4007F33D12D4B9B69B5
:1052600013F4806F04D02B4BDB6913F4806F29D1CA
:10527000284B9B6913F4807F04D0264BDB6913F421
:10528000807F2FD1234BDB6913F4805FBFD0214C8B
:105290004FF480532362254B9847254B984763680A
:1052A00023F001036360636823F002036360214B12
:1052B0009847214B98474FF4807323614FF4006364
:1052C0002361A4E7134C4FF4185323626361012058
:1052D0001A4B98474FF48073236223614FF40063A5
:1052E000236110BD0B4B4FF480721A625A614FF468
:1052F00000521A614FF400721A614FF480621A6111
:1053000030200F4B984700200C4B984710BD00BF32
:10531000E162400000400440A96140004951400062
:10532000FA010020153F4000A54B4000D94740003E
:105330003D3D400041424000F54240009D4140005B
:10534000FD61400010B582B0EFF31083B3FA83F330
:105350005B09019372B6BFF35F8F0022144B1A7082
:10536000019C0120134B98473020134B9847134B57
:105370005A6F22F480725A675A6F42F400725A6769
:105380004FF480721A614FF400521A614FF40072A8
:105390001A614FF480621A614FF400621A612CB1F5
:1053A0000122034B1A70BFF35F8F62B602B010BDCB
:1053B000FA0100209D414000A961400000400440E6
:1053C00030B583B0EFF31083B3FA83F35B09009336
:1053D00072B6BFF35F8F0024204B1C70009D204BE2
:1053E000984730201F4B98471F4B98471F4B502220
:1053F00083F830234FF480325A601D4B98474FF4A6
:1054000080201C4B98471C4B1C701C4B1B78FF2B9F
:1054100022D0EFF31083B3FA83F35B09019372B6E2
:10542000BFF35F8F00220D4B1A700199134A137856
:105430000133137029B10122084B1A70BFF35F8F3B
:1054400062B60F4B98472DB10122044B1A70BFF37F
:105450005F8F62B603B030BDFEE700BFFA010020E7
:10546000AD5B4000A9614000955D400000E100E0B7
:1054700061474000CD6240001D0D0020501B002000
:10548000455340000D4B5A6822F001025A609A6859
:1054900022F480729A60024670B1986820F07F0012
:1054A00002F07F02104398609A6842F480729A601A
:1054B0005A6842F001025A60704700BF0040044041
:1054C000054B5B6813F0010F04D0034B986800F0A4
:1054D0007F0070470020704700400440014B9860F7
:1054E00099817047381B0020F0B583B045B200F0B9
:1054F0000F00052873D801F00306044600F10C03E1
:105500003B4F57F8233013F4004F6BD1012E53D08B
:10551000031FDBB2012B54D94023934266DB461EA6
:1055200006EB8607334B03EB870303F11007B3F851
:1055300010E062F3090EA3F810E05B7C03F07F0338
:105540006FF345137B70002D3EDB294EB36A0122B9
:1055500082401343B362264B9B6A1A42FBD0244B12
:105560009E6A26EA02029A6200F10C0253F8223087
:105570000193019B43F04F030193019B23F40743E5
:1055800023F080030193002D23DB0A0202F4407212
:1055900042F40042019B1343019301990C30144BD8
:1055A00043F8201004F10C03114951F8233032EA7A
:1055B0000303F7D1012013E0B0B10328A8D10020E4
:1055C0000EE04FF40073A8E77B786FF383037B70E2
:1055D000BBE70A0202F4407242F40442DAE7002018
:1055E00003B0F0BD0020FBE70020F9E70020F7E75B
:1055F00000400440240D002000F00F03052B1ED8AE
:1056000010B582B019460E4C0C3354F82320019289
:10561000019A42F04F020192019A22F40042019253
:10562000019A44F8232001F10C03054A52F8233073
:1056300013F4004FF7D1034B984702B010BD7047E9
:10564000004004400548400000F00F00431E0528BC
:1056500015D803EB83039A000A4B13445B7C13F0C9
:10566000200F08D10C30084B53F8203013F0280FCE
:1056700003D00120704701207047002070470020B0
:10568000704700BF240D00200040044010B485B0D6
:1056900044B200F00F00052865D8421EEFF31083D6
:1056A000B3FA83F35B09039372B6BFF35F8F0021F4
:1056B000314B19700399002C14DB304A00F10C04B3
:1056C00052F824300293029B43F04F030293029B53
:1056D00043F020030293029B42F8243000238DF80C
:1056E00007302EE000F10C03244C54F8233013F063
:1056F000100F09D102EB82039C00214B23445B7CF9
:10570000C3F38103012BD8DD02EB820294001C4B12
:1057100023445A7C42F020025A74012303FA00F019
:10572000164B186121B30120134B1870BFF35F8F24
:1057300062B619E000BF9DF807300133DBB28DF887
:1057400007309DF80730DBB2132BF3D9012303FA9E
:1057500000F00A4B186169B10120074B1870BFF3C4
:105760005F8F62B600E0002005B05DF8044B704723
:105770000120F9E70120F7E7FA010020004004408A
:10578000240D002000F00F0005286CD830B583B040
:105790000246441E04EB84039900354B0B44597CAC
:1057A0006FF34511597400F10C03324951F823305D
:1057B00013F0200F59D000F10C0551F8253000935B
:1057C000009B43F04F030093009B23F020030093C2
:1057D000009B41F8253002F10C03264951F8233093
:1057E00013F0200FF7D10D468B6A012181400B4346
:1057F000AB62204B9B6A1942FBD01E4B9D6A25EA87
:10580000010199620C3053F820100191019941F087
:105810004F010191019921F008010191019943F88B
:10582000201002F10C03134951F8233013F0080F34
:10583000F7D104EB84039A000D4B13445B7C13F007
:10584000100F01D1012011E00949A20010198300B5
:105850000B44587C6FF3041058741444A300CB58C5
:105860009847012002E000207047012003B030BDBE
:10587000240D002000400440F0B583B000F00F0478
:10588000052C00F2A28047B2651E04F10C00554EB3
:1058900056F8200010F4004F00F09A8005EB8500C8
:1058A000514E06EB8000407C10F0200F40F09280BB
:1058B00004F10C004B4E56F8200010F0200F40F081
:1058C0008B80EFF31080B0FA80F04009009072B640
:1058D000BFF35F8F002645480670DDF800E005EB5A
:1058E0008500414E06EB8000407C10F0100F0AD07E
:1058F000BEF1000F72D001223C4B1A70BFF35F8FD4
:1059000062B6002062E005EB8500374E06EB8000B2
:10591000467C46F010064674BEF1000F05D0012605
:1059200032480670BFF35F8F62B6DFF8BCE005EB6C
:10593000850080000EEB00067260B3600022F2600A
:10594000089A4EF8002011B95BBB012000E001204D
:10595000254AA9004B1902EB83035B7C60F3861395
:105960000D4402EB85026FF3C7135374EFF31083FA
:10597000B3FA83F35B09019372B6BFF35F8F002222
:105980001A4B1A70019D0123A340164A1361002F80
:1059900009DB2DB30120154B1870BFF35F8F62B682
:1059A00014E00020D4E704F10C0352F8233013F084
:1059B000110FEED1012120460D4B98470028E8D069
:1059C000002120460A4B9847E3E7002003B0F0BDD2
:1059D0000020FBE70020F9E70020F7E70020F5E7CB
:1059E0000120F3E700400440240D0020FA010020CC
:1059F000E549400070B586B000F00F04052C00F2B8
:105A0000C98042B2EFF31083B3FA83F35B090593C5
:105A100072B6BFF35F8F00215F4B1970059B26465E
:105A20000125A5405D494D612BB101215A4B1970EB
:105A3000BFF35F8F62B6002A80F2948004F10C03FA
:105A4000564A52F8233013F0100F64D0002C49D07E
:105A5000032C47D004F10C0152F821300193019B33
:105A600043F04F030193019B23F010030193019B2B
:105A700042F8213006F10C03484A52F8233013F063
:105A8000100FF7D106F10C03444A52F8233013F0FB
:105A9000100FF7D104F10C0152F821300293029B50
:105AA00043F04F030293029B43F010030293029BC7
:105AB00042F8213000238DF8033006E000BF9DF846
:105AC00003300133DBB28DF803309DF80330DBB2D5
:105AD000132BF3D906F10C03304A52F8233013F09C
:105AE000100FF7D02D4A04F10C0152F82130039326
:105AF000039B43F04F030393039B23F01003039393
:105B0000039B42F8213006F10C03244A52F823305B
:105B100013F0100FF7D1214A04F10C0152F8213093
:105B20000493049B43F04F030493049B23F001036D
:105B30000493049B42F8213006F10C03174A52F8F3
:105B4000233013F0010FF7D1621E02EB82029100A5
:105B5000134B0B445A7C6FF383025A740AE02046BD
:105B6000104B984706F10C030C4A52F8233013F0FF
:105B7000420FF4D1094A936A2B439362074B9B6A05
:105B80001D42FBD0054A936A23EA0505956220462B
:105B9000054B984706B070BDFA0100200040044054
:105BA000240D00202948400005484000064BD3F84A
:105BB000142122F44062C3F81421D3F8202142F0CA
:105BC0000102C3F82021704700020E400B4619B1B4
:105BD000096801605B6843601AB113680361536828
:105BE0004361704721F0FE01C905C90D016270478C
:105BF00010B51E4B53F820402268536A13F0805FA3
:105C000011D00223C2F8203123684FF0FF32DA614D
:105C100000232375236913F0010F26D0636823B393
:105C20002046984710BD13F0006F13D00223C2F82E
:105C3000203123684FF00062DA61236913F0020F0C
:105C400003D0A3680BB12046984723680122C3F80C
:105C5000202110BD13F0007F07D0236913F0040F3B
:105C600003D0E3680BB12046984710BD880D002093
:105C700008B50020014B984708BD00BFF15B40000C
:105C800008B50120014B984708BD00BFF15B4000FB
:105C900070B505460E461446016001230B60214B8A
:105CA00099422BD00D20204B9847204B1D60237824
:105CB0001B0203F4FE43736063782BBB0022A378BE
:105CC0000BB142F00402E3780BB142F008022379F1
:105CD0000BB142F0100263791B0203F47063A179E7
:105CE000090389B20B431343B3652389C3F30E033E
:105CF000628943EA0243F36500230CE012200A4B59
:105D000098470A4B5D60D2E70222D8E705EB830291
:105D1000002151600133022BF8D900202861287539
:105D200070BD00BF00000340A9614000880D002045
:105D300012F0100F12D0C0F8B01012F0200F07D0E0
:105D4000C0F8D41012F0400F05D0C0F8C010704752
:105D5000C0F8D010F6E7C0F8C4107047C0F8B4100F
:105D600070470164704741647047C06C7047806C35
:105D70007047400900F5001000F2077040027047BC
:105D800040090B30704700F01F00012303FA00F0B8
:105D90007047000008B500200A4B98470A4B984707
:105DA0000028FBD0094B9847094A0A4BDA620A4B94
:105DB00098470028FBD00020084B9847084B98478D
:105DC00008BD00BF25614000496140008D61400071
:105DD000013FB80500040E4099614000AD624000EB
:105DE000C162400010B5A2B01848194B9847002076
:105DF000184B9847184B98470028FBD0174B9847EB
:105E0000174A184B9A62184B98470028FBD000207D
:105E1000164B9847164B984716480D4B9847164B0C
:105E20001A68164B1344164A934201D922B010BD8A
:105E30002023009302AB0F220E211248124CA047E0
:105E4000BDF848101148124B9847EFE7000E27079E
:105E500019664000256140004961400071614000C1
:105E6000013FB70B00040E407D614000D16040004F
:105E7000256540000000DC05FC010020C0D3BDF911
:105E800080C3C901000A0E400100002010140E401A
:105E9000F162400070B50D461446064658B14FF009
:105EA000FF360AE0064B1868064B1B6829469847E0
:105EB00001350136013C002CF4DC304670BD00BFDA
:105EC000601B0020581B002070B5013802280FD835
:105ED000144600258CB10A4B18684E1C094B1B68F0
:105EE00009789847002806DB0135013C3146F1E787
:105EF0004FF0FF3501E04FF0FF35284670BD00BF81
:105F0000601B00205C1B0020A1F10E03012B02D8B6
:105F10004FF0FF30704710B582B0EFF31083B3FA43
:105F200083F35B09019372B6BFF35F8F00240B4BC1
:105F30001C70019C120222F07F4222F0FF02C9B2C3
:105F4000114341F0B441064B98472CB10122034B59
:105F50001A70BFF35F8F62B602B010BDFA01002065
:105F6000690000204C4B1B78FF2B31D000B583B06B
:105F7000EFF31083B3FA83F35B09019372B6BFF3B7
:105F80005F8F0022454B1A700199434A1378013301
:105F9000137029B10122414B1A70BFF35F8F62B6B3
:105FA0003F4A904215D03F4A904220D03E4A90420C
:105FB0002BD03E4A904236D03D4A904241D03D4A95
:105FC00090424CD03C4A904257D003B05DF804FB5D
:105FD000FEE71620394B98470720394B9847002198
:105FE0000720384B98470720374B9847EDE7152097
:105FF000324B98470720324B984700210720314BFE
:1060000098470720304B9847DFE714202B4B9847E1
:1060100007202B4B9847002107202A4B9847072041
:10602000294B9847D1E71320244B98470620244B4F
:10603000984700210620234B98470620224B98477B
:10604000C3E70E201D4B984706201D4B98470021A3
:1060500006201C4B984706201B4B9847B5E70920A4
:10606000164B98470620164B984700210620154BE3
:1060700098470620144B9847A7E708200F4B9847EE
:1060800006200F4B9847002106200E4B984706200C
:106090000D4B984799E700BF501B0020FA010020E4
:1060A000000004400080004000C00140008001402A
:1060B000004002400000024000C00040A9614000D2
:1060C0009962400051624000856240000160704763
:1060D000134A136B23F07003184310634FF40063EB
:1060E0000F4A926E12F0080F02D1A3B1013BF7E7FD
:1060F0000B4A136B23F0030343F0020313634FF4C3
:106100000063074A926E12F0080F02D12BB1013BD7
:10611000F7E700207047012070470120704700BF5B
:1061200000040E40012803D0054A064B1A60704750
:10613000044A936843F0254343F480139360F3E7E4
:10614000080000A510140E40074B5B6913F0800F88
:1061500006D0064B9B6E13F0800F03D100207047D2
:10616000002070470120704710140E4000040E40BC
:106170000022014B9A62704700040E40024B986E59
:1061800000F00200704700BF00040E400022014BE7
:10619000DA62704700040E40024B986E00F0040073
:1061A000704700BF00040E4032281ED81F280CD8AC
:1061B000114B9A6901238340934318D0012303FABA
:1061C00000F00D4B18610020704720380A4BD3F8BF
:1061D00008210123834093430BD0012303FA00F0ED
:1061E000054BC3F8000100207047012070470020D4
:1061F00070470020704700BF00040E40322822D8AC
:106200001F280ED8114B9A6901238340934301D074
:1062100000207047012303FA00F00C4B5861002066
:1062200070472038094BD3F808210123834093435A
:1062300001D000207047012303FA00F0034BC3F89C
:106240000401002070470120704700BF00040E4089
:1062500041F0040100F11002094B43F822104FF401
:106260000062074B996E4FF480738340194202D14C
:106270001AB1013AF5E7002070470120704700BFCE
:1062800000040E404FF4807303FA00F0014B1860D5
:10629000704700BF00040E404FF4807303FA00F013
:1062A000014B5860704700BF00040E40000200F42C
:1062B000706040F00100014B9863704700040E408D
:1062C0008022014B1A60704700040E40C0F3120098
:1062D000024B1A6F10431867704700BF00040E404E
:1062E000024B187880F00100704700BF900D00202D
:1062F000C36923F4F053490201F4F051194341F00A
:10630000B44141F48071C161704730B4B2EB011FF8
:1063100017D3102401FB04F14B0803EBC202B2FBBC
:10632000F1F2D3085D1E4FF6FE718D4210D8082C95
:1063300009D0120402F4E0221A430262002030BCA9
:1063400070470824E6E7416841F400214160F0E726
:106350000120F4E7402303607047882303607047FF
:106360001023036070472423036070474FF4807349
:10637000036070474FF4002303607047436913F0D4
:10638000020F04D0C1F30801C16100207047012051
:106390007047436913F0020FFBD0C1F30801C161DC
:1063A00000207047436913F0010F05D08369C3F3E0
:1063B00008030B600020704701207047014BC0F8B4
:1063C000E43070470041535510B50446094B9847D7
:1063D000002363606362A3622046074B9847204610
:1063E000064B98472046064B98472046054B984752
:1063F00010BD00BFBD6340005B63400067634000A9
:106400006D6340007563400070B505460C46164646
:10641000104B98470022104B1A60B4B132462168E5
:1064200028460E4B9847024688B96368A1680B431B
:1064300021690B43E1680B430749086803430B607C
:1064400069680B436B60104670BD0122FBE70122B7
:10645000F9E700BFC9634000940D00200B634000C2
:10646000FEE7000000B583B0234B244A9A4209D0CE
:10647000214B224A03E01168196004330432204999
:106480008B42F8D31F4B02E000221A6004331E4AED
:106490009342F9D31D4A22F07F011D4B9960EFF31F
:1064A0001083B3FA83F35B09019372B6BFF35F8F76
:1064B0000021184B1970019817490B6843F47003B9
:1064C0000B60BFF34F8FBFF36F8F28B10121114BCA
:1064D0001970BFF35F8F62B602F16042B2F5203FE0
:1064E00004D20B4A936843F0005393600B4B9847D8
:1064F0000B4B9847FEE700BF00000020D0C34000D0
:10650000B80B0020B80B0020B41B00200000400096
:1065100000ED00E0FA01002088ED00E02D8E400043
:106520002D7E4000344B1B6B03F00303012B20D066
:1065300083B1022B39D0304B1B6B03F07003702BEF
:1065400051D02D4B1A6BC2F302122C490B68D34069
:106550000B6070472A4B5B6913F0800F04D04FF437
:106560000042264B1A60E6E74FF4FA42234B1A60CA
:10657000E1E7214B1B6A13F0807F03D0214A1F4BB8
:106580001A60D8E7204A1D4B1A601B4B1B6A03F0A8
:106590007003102B05D0202BCDD11C4A174B1A604D
:1065A000C9E71B4A154B1A60C5E7154B5B6913F029
:1065B000800F13D04FF40042104B1A600E4B1B6B30
:1065C00003F00303022BB6D10B4B9A6AC2F30C42C1
:1065D0000A490B6802FB03330B60ACE74FF4FA4245
:1065E000064B1A60EAE7054A13680A49A1FB031340
:1065F0005B081360704700BF00040E40FC010020E0
:1066000010140E40001BB70000127A0000366E0115
:106610000024F400ABAAAAAA144B98420FD9144B39
:10662000984211D9134B984212D9134B984213D95F
:10663000124B984214D9124A124B1A6070474FF00D
:106640008062104B1A6070470F4A0E4B1A607047F9
:106650000E4A0C4B1A6070470D4A0A4B1A6070477D
:106660004FF00422074B1A60704700BFFF2C310126
:10667000FF596202FF869303FFB3C404FFE0F505F0
:1066800000050004000A0E4000010004000200049E
:10669000000300040A4B1B6853B1094B1B681A180E
:1066A0000849914208DB1046054A106018467047B9
:1066B000054A034B1A60F0E74FF0FF30704700BF08
:1066C000980D0020FC7F0220B84B00204FF0FF30D7
:1066D00070474FF400534B60002070470120704713
:1066E0000020704700F1080343604FF0FF328260E2
:1066F000C360036100230360704700230361704798
:1067000043684B609A688A609A6851609960086132
:10671000036801330360704730B40D68B5F1FF3F83
:1067200002D000F1080202E0026904E01A46536850
:106730001C68A542FAD253684B6099608A60516028
:10674000086103680133036030BC70470369426825
:10675000816891608268416851605A68904206D0B1
:10676000002202611A68013A1A601868704782684C
:106770005A60F5E782B0002301934FF0500383F392
:106780001188BFF36F8FBFF34F8F019B002BFCD09D
:1067900002B0704708480068006880F308884FF02E
:1067A000000080F3148862B661B6BFF34F8FBFF369
:1067B0006F8F00DF00BF000008ED00E0DFF80C0085
:1067C000016841F4700101607047000088ED00E04D
:1067D0004FF0807340F8043C21F0010140F8081CA0
:1067E000054B40F80C3C40F8202C6FF0020340F8B9
:1067F000243C4438704700BF75674000000000002B
:10680000074B19680868B0E8F04F80F30988BFF3B8
:106810006F8F4FF0000080F311887047AFF3008056
:106820009C0D00204FF0500383F31188BFF36F8F4E
:10683000BFF34F8F024A136801331360704700BFE4
:1068400000020020034A1368013B13600BB983F375
:1068500011887047000200200000000000000000C6
:10686000EFF30980BFF36F8F154B1A681EF0100FFE
:1068700008BF20ED108A20E9F04F10602DE90900D3
:106880004FF0500080F31188BFF34F8FBFF36F8F2D
:1068900000F03CFE4FF0000080F3118809BC19683D
:1068A0000868B0E8F04F1EF0100F08BFB0EC108A77
:1068B00080F30988BFF36F8F704700BFAFF300808C
:1068C0009C0D002008B54FF0500383F31188BFF3EF
:1068D0006F8FBFF34F8F054B984718B14FF0805221
:1068E000034B1A60002383F3118808BD89724000AE
:1068F00004ED00E0054B00221A6005490A600549D5
:10690000054A116007221A60704700BF10E000E0DE
:1069100018E000E0FF7F010014E000E010B50E4B2E
:106920001A6842F470021A601A6842F070421A60E3
:106930000A4B984700240A4B1C600A4B98470A4AA6
:10694000136843F040431360084B9847084B98473F
:10695000084B9847204610BD20ED00E0F568400048
:1069600000020020BD67400034EF00E09567400062
:106970000D7540007567400010B50446044B9847FC
:106980002046044B98470446034B9847204610BDC9
:1069900079724000A58E40007D73400048B110B56B
:1069A0000446044B98472046034B9847034B9847AF
:1069B00010BD704779724000B58E40007D73400075
:1069C000436A23B1036B1868C0F1050070470020CB
:1069D0007047000010B50446064B9847A26BE36B66
:1069E0009A4204D00024044B9847204610BD01244D
:1069F000F9E700BF256840004568400010B504462F
:106A0000054B9847A36B23B10024044B98472046BD
:106A100010BD0124F9E700BF25684000456840002B
:106A200070B504461646856B026C5AB903681BB1F3
:106A300000200135A56370BD4068174B98470023BF
:106A40006360F6E76EB98068144B9847226CA368C0
:106A50001344A3606268934219D32368A3600020A3
:106A6000E7E7C0680D4B9847226C5242E368134435
:106A7000E36021688B4202D263681A44E260022E0E
:106A800001D00020D5E725B1013D0020D1E700204D
:106A9000CFE70020CDE700BFC1774000D194400090
:106AA00038B505461A4B984795F8454064B201E061
:106AB000013C64B2002C0ADD6B6A43B105F124008D
:106AC000144B98470028F3D0134B9847F0E7FF2367
:106AD00085F84530114B98470D4B984795F8444041
:106AE00064B201E0013C64B2002C0ADD2B6943B1C1
:106AF00005F11000074B98470028F3D0064B984744
:106B0000F0E7FF2385F84430044B984738BD00BFB9
:106B100025684000E5754000E1764000456840008A
:106B200038B504460D46144B98472168E26B236C38
:106B300003FB021060600020A063A160013A02FB29
:106B40000313E360FF2384F8443084F8453055B9DB
:106B500023691BB9094B9847012038BD04F1100087
:106B6000074B9847F6E704F11000064DA84704F1DB
:106B70002400A847EEE700BF2568400045684000B4
:106B8000E5754000E566400038B51D46049C0B469F
:106B900049B12260E063236401212046034B9847FA
:106BA00084F84C5038BD2460F4E700BF216B4000EE
:106BB000F0B583B0054617460E4689B100FB01F0DB
:106BC0005030084B9847044638B100903B4600F1DE
:106BD000500231462846044DA847204603B0F0BD78
:106BE0000020EDE779694000896B4000F0B585B081
:106BF00004460F4601921E46002526E032463946DD
:106C00002046354B9847636A23B9344B9847012097
:106C100005B0F0BD04F12400314B9847F5E72F4B48
:106C200098470020F4E702A82E4B9847012519E069
:106C3000002384F8443021E0002384F8453023E029
:106C40002046294B9847294B9847294B9847A26BD8
:106C5000E36B9A42D2D3022ED0D0019B002BDED020
:106C6000002DE0D01D4B9847224B9847204B98476A
:106C700094F844305BB2B3F1FF3FD9D094F845307B
:106C80005BB2B3F1FF3FD7D0144B984701A902A8DC
:106C9000194B9847C8B92046184B98470028CFD0C1
:106CA000019904F11000164B984720460E4B984767
:106CB0000E4B98470028C8D14FF08052114B1A60F4
:106CC000BFF34F8FBFF36F8FBFE72046064B984748
:106CD000064B984700209BE7216A4000456840002A
:106CE000E575400065764000A16A40007D73400074
:106CF00025684000797240007D764000D5694000EB
:106D0000C175400004ED00E048B110B500214160BC
:106D10000160C1600B460A46014CA04710BD704798
:106D2000ED6B400010B5024600210120034B98474F
:106D30000446034B9847204610BD00BFB16B40008E
:106D4000096D400070B584B00446019100263546B7
:106D50003EE0013BA36323683BB123694BB9444B3D
:106D600098470126304604B070BD424B984760609A
:106D7000F3E704F11000404B9847F0E73C4B98478D
:106D80000026EFE702A83D4B984701252AE00023A3
:106D900084F8443032E0002384F8453034E0384B46
:106DA00098476068374B98470646314B98473BE019
:106DB0002046354B9847354B984709E02046324BE3
:106DC0009847324B98472046314B9847002840D18E
:106DD0002B4B9847A36B002BBBD1019B002BCDD035
:106DE000002DCFD0224B98472A4B9847244B9847E9
:106DF00094F844305BB2B3F1FF3FC8D094F845300B
:106E00005BB2B3F1FF3FC6D0194B984701A902A866
:106E1000214B98470028D1D120461D4B9847002888
:106E2000C6D02368002BBAD0019904F124001B4B73
:106E300098472046144B9847144B98470028C7D1D1
:106E40004FF08052164B1A60BFF34F8FBFF36F8F16
:106E5000BEE7002E86D00A4B98472046114B984734
:106E600001466068104B9847014B9847002679E728
:106E700045684000E9784000E575400065764000CF
:106E800025684000F9764000A16A40007D7340000B
:106E9000FD694000797240007D764000C175400078
:106EA00004ED00E0C169400049784000F0B5036896
:106EB0004BB343685B68436000F10807BB4204D0F2
:106EC0004368D3F80CE0002609E05B684360F7E70D
:106ED0005B68436008E02E46B6B9AE4514D04368FF
:106EE0005B6843609F42F3D04368DD6800230F2B4B
:106EF000F2D8EA1892F83420CC5CA242ECD1002AF5
:106F0000E9D00133F3E700263046F0BD0A4B1B6899
:106F10001B684BB901234BB9074B1B68DB68DB6867
:106F20005A68064B1A6070470023F4E74FF0FF32AF
:106F3000024B1A60704700BFA00D00204C0E0020CD
:106F40002DE9F84F81460D4617469A460A9EDDF810
:106F50002C800C9C9200A521206B1D4B9847236B25
:106F600007F18042013A03EB820727F0070700236D
:106F70000F2B07D8E95CE21882F83410EA5C0AB1FA
:106F80000133F5E7002384F84330042E00D90426AA
:106F9000E662E66400252565201DDFF83CB0D84791
:106FA00004F11800D8472461C6F10506A6616462A1
:106FB000656584F85850524649463846054B98470F
:106FC0002060B8F1000F01D0C8F80040BDE8F88F8C
:106FD000CD964000D1674000FB66400070B50024AC
:106FE00007E004EB840293000B4818440B4B9847CE
:106FF0000134042CF5D90A4E3046084CA047094DFF
:107000002846A0470848A0470848A047084B1E60EC
:10701000084B1D6070BD00BFA80D0020E566400054
:10702000200E0020340E0020540E00206C0E002094
:10703000A00D0020A40D002010B504461C4B98475D
:107040001C4A1368013313601B4B1B68002B26D0AE
:107050001A4B1B683BB9184B1B68DA6AE36A9A4201
:1070600001D8154B1C60164A136801331360636422
:10707000E36A01229A401349086802430A6003EB5D
:1070800083039A00211D10481044104B9847104B61
:1070900098470A4B1B680BB1074B1B6810BD064B8A
:1070A0001C601368012BDED10A4B9847DBE700BF59
:1070B000256840000C0E00209C0D0020680E00206A
:1070C000180E00201C0E0020A80D002001674000B3
:1070D00045684000DD6F400070B504460E461D4B0C
:1070E0001D681D4B186804301C4B984750B91A4B4B
:1070F0001B68DA6A012303FA02F219490B6823EAD2
:1071000002030B60B4F1FF3F13D02C44124B1B68F9
:107110005C60A54216D8134B18680F4B19680431F0
:10712000114B9847114B1B689C4201D20F4B1C60BE
:1071300070BD002EE9D0084B196804310C480D4B86
:10714000984770BD0C4B1868034B19680431064B07
:10715000984770BD800E00209C0D00204D674000B8
:107160001C0E0020A00D0020196740004C0E0020CE
:107170006C0E002001674000A40D002008B54FF000
:107180008052044B1A60BFF34F8FBFF36F8F024BD7
:107190009847F4E704ED00E0297E40002DE9F04334
:1071A00085B006460F46154698469000144B984702
:1071B00000B381465C20124B98470446B0B1C0F83A
:1071C0003090CCB10023039302940D9B01930C9B50
:1071D000009343462A46394630460A4DA847204682
:1071E000094B9847012005B0BDE8F0834846074B9E
:1071F0009847E6E70024E4E74FF0FF30F3E700BFED
:1072000079694000416F4000397040009D6940003D
:1072100010B582B0104B01930023009346220F4912
:107220000F48104CA047012801D002B010BD4FF00C
:10723000500383F31188BFF36F8FBFF34F8F4FF06D
:10724000FF32094B1A600122084B1A600022084BDA
:107250001A60084B9847E8E7480E002070C14000CC
:107260007D7140009D7140004C0E0020680E002092
:10727000800E00201D694000024A1368013313602C
:10728000704700BF140E002070B52F4B1B68002BF9
:1072900052D12E4B1E6801361E604EB12C4B1B681E
:1072A0009E422FD22B4B1B68002B42D0002070BD7A
:1072B000294A1168294B186810601960284A136818
:1072C00001331360274B9847E8E7012320E04FF094
:1072D000FF321F4B1A60E5E71D4A1360E2E704F135
:1072E0001800214B9847E36A01229A401F49086819
:1072F00002430A6003EB83039A0029461C481044AA
:107300001C4B9847144B1B681B68002BDDD00023D7
:10731000002BDCD1104B1B68DB68DC6863689E4285
:10732000DAD3251D2846104B9847A36A002BD6D1E7
:10733000D9E7114B9847B9E7064A13680133136040
:107340000D4B9847B2E700BF140E0020800E0020BE
:107350004C0E0020100E0020A00D0020A40D0020D7
:10736000500E00200D6F40004D6740001C0E0020A5
:10737000A80D0020016740002B7E400070B5274B10
:107380009847274B1A68013A1A601B68002B32D1C4
:10739000244B1B68002B2ED00024234B1B6813B3F7
:1073A000214BDB68DC6804F11800204EB047251D36
:1073B0002846B047E36A01229A401D490868024303
:1073C0000A6003EB83039A0029461A4810441A4BBB
:1073D0009847E26A194B1B68DB6A9A42DDD30122A7
:1073E000174B1A60D9E70CB1164B9847164B1C681F
:1073F0003CB9134B1B68154B9847002070BD013CEE
:1074000007D0134B98470028F9D001220C4B1A6083
:10741000F5E700220C4B1A60EBE700BF256840003F
:10742000140E00200C0E0020540E00204D6740006A
:107430001C0E0020A80D0020016740009C0D0020BC
:10744000840E00200D6F4000100E002045684000A3
:107450008972400010B550B9002038B94FF0805201
:10746000084B1A60BFF34F8FBFF36F8F10BD0446F8
:10747000054B984700212046044B9847044B9847FA
:10748000EBE700BF04ED00E079724000D9704000E6
:107490007D73400070B50646154B98470524013CA6
:1074A00004EB84029300314612481844124B98476B
:1074B000054608B9002CF2D12DB15DB18DB10F4B4D
:1074C0009847284670BD0E4B186831460A4B9847BE
:1074D0000546F2E70B4B18683146074B98470546BF
:1074E000ECE731460848044B98470546E7E700BFFC
:1074F00079724000A80D0020AD6E40007D73400001
:10750000A00D0020A40D00206C0E0020264B1B684F
:10751000002B2FD110B50022244B1A60244B1B687E
:107520001B6B1A68B2F1A53F28D0214B1868196867
:107530003431204B9847204B1B68B3FA83F3DBB2FE
:10754000C3F11F031D489A00D418A10001444C68E0
:1075500064684C601A4491000831084484421AD08F
:1075600003EB83039A00154B13445B68DA68104BF6
:107570001A6010BD01220D4B1A6070475A68B2F1B3
:10758000A53FD2D19A68B2F1A53FCED1DB68B3F165
:10759000A53FCAD1CFE7606803EB83029100074A99
:1075A0000A445060DCE700BF140E0020840E002067
:1075B0009C0D0020117E40001C0E0020A80D002014
:1075C00010B50C46044B19681831044B984701213B
:1075D0002046034B984710BD9C0D002019674000C2
:1075E000D970400038B5C368DC6804F11805284636
:1075F000144B9847144B1B68E3B9251D2846114BC3
:107600009847E36A01229A401049086802430A60D9
:1076100003EB83039A0029460D4810440D4B98470D
:10762000E26A0D4B1B68DB6A9A4208D901200B4BBA
:10763000186038BD29460A48064B9847F0E70020F5
:1076400038BD00BF4D674000140E00201C0E002006
:10765000A80D0020016740009C0D0020840E002032
:10766000540E0020034B1B680360034B1B684360F0
:10767000704700BF500E0020800E0020F8B5044671
:107680000D46124B9847124B19686268881A2B688E
:10769000B3F1FF3F16D027680E4E3668B74201D0CF
:1076A000914211D2984206D300232B6001240A4B49
:1076B00098472046F8BD1B1A2B602046074B984779
:1076C0000024F4E70024F2E70124F0E725684000F5
:1076D000800E0020500E0020456840006576400076
:1076E0000122014B1A607047840E0020014B18687C
:1076F000704700BF9C0D0020002854D038B50446C8
:10770000C26A2A490968C96A8A4242D28169002943
:1077100005DB26490968C96AC1F105018161606913
:1077200002EB82029100224A0A44904207D00022D2
:107730003AB91E4A1268D26AE262012038BD0122BB
:10774000F6E7251D28461B4B984768B9E36A03EB0B
:1077500083018A0016498A5832B901229A40164993
:107760000B6823EA02030B60104B1B68DB6AE362C1
:10777000012404FA03F21049086802430A6003EB8B
:1077800083039A0029460A4810440C4B9847204628
:1077900038BDC26C054B1B68DB6A9A4201D20120DE
:1077A00038BD002038BD0020704700BF9C0D002070
:1077B000A80D00204D6740001C0E0020016740000E
:1077C000002834D038B50446026D013A0265C06A1B
:1077D000E16C88422DD00AB1002038BD251D284615
:1077E000154B984768B9E36A03EB83018A00134994
:1077F0008A5832B901229A4011490B6823EA0203E0
:107800000B60E36CE362C3F10502A261012404FA98
:1078100003F20B49086802430A6003EB83039A00F2
:10782000294606481044074B9847204638BD00209B
:107830007047002038BD00BF4D674000A80D0020F4
:107840001C0E002001674000002843D038B50446D4
:10785000C26C8A4200D20A46E16A8A4202D0206D96
:10786000012800D038BDE262A069002802DBC2F125
:107870000502A261636901EB81018800164A024496
:10788000934225D00022002AECD0251D2846134B18
:10789000984768B9E36A03EB83018A000E498A5866
:1078A00032B901229A400E490B6823EA02030B60A9
:1078B000E36A01229A400A49086802430A6003EB1E
:1078C00083039A00294604481044064B9847C9E7A9
:1078D0000122D8E7704700BFA80D00204D67400087
:1078E0001C0E002001674000054B1B6823B1044BB0
:1078F0001A68136D01331365014B1868704700BF98
:107900009C0D002038B505460C461A4B98471A4B7B
:107910001B685B6D2BB9184B1B68012283F858203C
:10792000ACB9164B9847134B9847134B1B685C6DCB
:1079300024B1CDB9104B1B68621E5A650E4B1B68F3
:10794000002283F858200D4B9847204638BD114639
:1079500020460B4B98474FF080520A4B1A60BFF3FA
:107960004F8FBFF36F8FDCE7034B1B6800225A6514
:10797000E4E700BF256840009C0D002045684000FA
:10798000D970400004ED00E0F8B5EFF311854FF039
:10799000500484F31188BFF36F8FBFF34F8F0BB187
:1079A000446D1C6090F85830DBB2022480F85840D7
:1079B000013A032A1AD8DFE802F0020C1114426DD2
:1079C000114341650126012B14D085F311883046FF
:1079D000F8BD426D013242650126F4E7416501269A
:1079E000F1E7022B04D041650126ECE70126EAE726
:1079F0000026E8E70446164B1B68F3B9071D384616
:107A0000144B9847E36A01229A40134908680243DD
:107A10000A6003EB83039A00394610481044104B68
:107A20009847E26A0F4B1B68DB6A9A42CDD9069BE6
:107A30004BB10123069A1360C7E700F118010A4809
:107A4000074B9847EDE70122084B1A60BDE700BFDE
:107A5000140E00204D6740001C0E0020A80D0020D1
:107A6000016740009C0D0020540E0020840E002071
:107A7000F8B5EFF311854FF0500383F31188BFF38E
:107A80006F8FBFF34F8F90F85830DBB2022280F82F
:107A90005820426D01324265012B02D085F31188D6
:107AA000F8BD0E460446154B1B68E3B9071D384662
:107AB000134B9847E36A01229A401249086802432F
:107AC0000A6003EB83039A0039460F4810440F4BBA
:107AD0009847E26A0E4B1B68DB6A9A42DED946B1D0
:107AE00001233360DAE700F118010A48074B984791
:107AF000EFE70122084B1A60D0E700BF140E002008
:107B00004D6740001C0E0020A80D002001674000BA
:107B10009C0D0020540E0020840E0020064BDB6BD1
:107B2000C3F30023054A1370054BDB6BC3F34033EB
:107B3000044A1370704700BF00100E40880E0020EA
:107B4000000E0E40890E002008B5054BDB6B13F4C8
:107B5000004F02D1034B984708BD034B984708BD1F
:107B6000000E0E40910A4000B50A400030B583B0C7
:107B700004460D46002301932E4B984213D02E4B02
:107B80009C421AD02D4B9C4221D02D4B9C4228D098
:107B90002C4B9C422FD02C4B9C4236D02B4B9C42E2
:107BA0003DD003B030BD01A92046294B984700289D
:107BB000F9D19DF804302B70E1E701A92046244B50
:107BC00098470028F9D19DF804302B70DAE701A915
:107BD00020461F4B98470028F9D19DF804302B70A0
:107BE000D3E701A920461A4B98470028F9D19DF800
:107BF00004302B70CCE701A92046154B984700288C
:107C0000F9D19DF804302B70C5E701A92046104B2F
:107C100098470028F9D19DF804302B70BEE701A9E0
:107C200020460B4B98470028F9D19DF804302B7063
:107C3000B7E700BF00C2004000020240004202401D
:107C40000082014000C20140008200400002044066
:107C5000A563400038B504460D46274B984213D023
:107C6000264B984218D0264B98421DD0254B98425F
:107C700022D0254B984227D0244B98422CD0244B1D
:107C8000984231D0002038BD29462046214B9847E4
:107C90000028F9D1012038BD294620461D4B9847C0
:107CA0000028F9D1012038BD29462046194B9847B4
:107CB0000028F9D1012038BD29462046154B9847A8
:107CC0000028F9D1012038BD29462046114B98479C
:107CD0000028F9D1012038BD294620460D4B984790
:107CE0000028F9D1012038BD29462046094B984784
:107CF0000028F9D1012038BD00C200400002024036
:107D0000004202400082014000C201400082004067
:107D1000000204407D63400000B583B002A9002347
:107D200041F8043D084B1868084B9847019B3BB14C
:107D30004FF08052064B1A60BFF34F8FBFF36F8F27
:107D400003B05DF804FB00BF8C0E0020717A400088
:107D500004ED00E070B58AB01D4B0FCB0AAC04E90E
:107D60000F001C4D1C4B1D601C4A1D4B1A601D4A08
:107D70001D4B1A60069B0093079B0193089B02937F
:107D8000099B039300240494184E3046184B9847DF
:107D900001213046174B9847174A69462846174B2A
:107DA00098472846164B98472846164B9847164E34
:107DB000336821469868154DA847336821465868AE
:107DC000A847336821469868A8470AB070BD00BF2D
:107DD00078C1400000820140601B0020557C4000BB
:107DE0005C1B00206D7B4000581B00200080014080
:107DF000655F4000CD6040000000DC050964400084
:107E0000556340006163400008020020A5974000D0
:107E100008B50A4601460248024B9847FEE700BFF4
:107E20001CC240007D8E4000704770472DE9F04332
:107E300083B0554B9847554A936843F0254343F424
:107E400080139360524B9847524B98470120524BF6
:107E50009847524B98470446514B9847002800F0EA
:107E6000908094F89930002B40F0878094F89740E8
:107E70004C4B98474C4B98474C4B98474C4B98472A
:107E800005464C4B9847F022014628464A4B9847F6
:107E90004A4B98474A4B984720464A4B98474A488E
:107EA0004A4B03602223037123234371484D294623
:107EB000484CA0474848494B03602B2303712A23B1
:107EC00043712946A047464B9847464B984746483A
:107ED000464B98474648474CA04747494748A04724
:107EE000474A48494848A04700230193042200928A
:107EF0004FF4807245494648464CA047012802D0BD
:107F000045483C4B98474148444B9847444B186080
:107F1000444B9847444B9847444A00210F20444E15
:107F2000B047444C03220B212046434DA847DFF8BD
:107F300018914A4600212820B047404F03220C21C7
:107F40003846A8472820DFF80481C0470146384654
:107F50003B4FB8474A4600210D20B04703220B2172
:107F60002046A8470D20C04701462046B847354B5C
:107F70009847002003B0BDE8F0830020064B9847E7
:107F800074E7502474E700BFD503400010140E407E
:107F9000E55D400029284000850A4000051B40009F
:107FA000D91B4000910A4000557D40002D3540000E
:107FB000953640009D364000A5354000C135400053
:107FC00029094000D9094000781B00200000024028
:107FD000A0860100AD244000641B002000C00140C9
:107FE000313D4000B5014000197D4000C90340000B
:107FF00088C140007D8E4000A4C14000B8C140004F
:10800000C0C14000CCC14000D8C14000F0C1400018
:10801000A93640009D714000F8C1400095744000B1
:108020008C0E0020C12F400029204000497B4000D9
:1080300081404000000E0E40F140400000100E4014
:10804000635D4000117240001D7B4000875D400071
:1080500000487047781B002000487047641B0020D0
:1080600008B5014B984708BDA536400008B5014B3F
:10807000984708BDA73640000120704708B5024860
:10808000024B984708BD00BF781B0020A125400087
:1080900008B50248024B984708BD00BF641B00208A
:1080A000A1254000014B1878704700BF890E0020C1
:1080B000014B1878704700BF880E002070B58AB059
:1080C000044600F06FF8324B93F900506B1C0646E3
:1080D00009D02146204600F08DFE20B9002120461F
:1080E00000F07EFE10B130460AB070BD294B0890FA
:1080F0002046019300F006FBCDE90401CDE9020121
:108100002046CDB9244B4FF060420021CDE9062333
:1081100000F03EFE002833D002230093684600F0B2
:1081200085F9A8B1089BC3B9DDE9060100F03EFB63
:10813000064630460AB070BD184B00220021CDE93A
:10814000062300F025FE68B102239D420093E5D18D
:1081500000F066FE22230360E4E700F061FE089B66
:108160000360E1E70123022D00930BD100F058FEDC
:10817000212303600A4800F05BF9CDE90601D1E74D
:1081800001230093684600F051F90028F2D1EDE791
:108190000402002034C24000FFFFEFC70000F0FFE0
:1081A000A0C140002DE9F84F30F000432DD0002849
:1081B000014604464ADBB0F1FF4F3BDAB0F5000F51
:1081C0003CDB00268D4AC4F316052A4402F4000263
:1081D000E41582F07E507F3C34444FF07E512843BA
:1081E00004EBD25400F036FB05F10F03C3F3160382
:1081F0000F2B064631DC002100F0CAFD002800F0FC
:1082000094804CB90020BDE8F88F00214FF04C401D
:1082100000F0DEFCBDE8F88F204600F0D1FB784985
:10822000054600F021FC77490446284600F01CFC76
:108230000146204600F010FBBDE8F88F4FF0984152
:1082400000F012FC6FF018060446BBE700F002FBDA
:10825000002100F0BDFCBDE8F88F4FF0804100F038
:10826000FBFA0146304600F0B3FC8046204600F0A1
:10827000A7FB41468146404600F0F6FB0146834697
:1082800000F0F2FB6049DFF8A0A1074600F0ECFB2C
:108290005E4900F0E1FA394600F0E6FB5C4900F087
:1082A000DBFA394600F0E0FB5A4900F0D5FA5946AE
:1082B00000F0DAFB58498346384600F0D5FB5749B1
:1082C00000F0CAFA394600F0CFFB554900F0C4FA75
:1082D000394600F0C9FB0146584600F0BDFAC5F525
:1082E0005713AA4403F5227343EA0A03002B0746F7
:1082F00065DD4FF07C51304600F0B6FB314600F0B2
:10830000B3FB0546002C32D12946384600F0A4FACA
:10831000414600F0A9FB0146284600F09BFA0146C1
:10832000304600F097FABDE8F88F3E49304600F03D
:108330009BFB01464FF07C5000F08CFA314605461D
:10834000304600F091FB0146284600F08DFB0546C3
:10835000002C2ED0204600F033FB2949074600F0C0
:1083600083FB28490446384600F07EFB14E024498C
:10837000484600F079FB29460446384600F06CFA7E
:10838000414600F071FB1F490746484600F06CFB70
:108390000146384600F060FA0146284600F05AFAD5
:1083A000314600F057FA0146204600F053FABDE886
:1083B000F88F0146304600F04DFABDE8F88F7CB1E9
:1083C0000F49484600F050FB39460446304600F05D
:1083D00041FA414600F048FB0A4905464846C3E7D2
:1083E0000146304600F036FA414600F03DFB0146BA
:1083F000304600F02FFABDE8F88F00BF20FB4A009E
:108400008071313FD1F717379788173E25333A3EB1
:108410002549923EABAA2A3F4FD01C3E298E633E8F
:10842000CDCCCC3EABAAAA3E305CCFFF002070473B
:1084300000200149704700BF0000F87F81F0004133
:1084400002E000BF83F0004330B54FEA41044FEA39
:10845000430594EA050F08BF90EA020F1FBF54EAD4
:10846000000C55EA020C7FEA645C7FEA655C00F070
:10847000E2804FEA5454D4EB5555B8BF6D420CDD41
:108480002C4480EA020281EA030382EA000083EAC4
:10849000010180EA020281EA0303362D88BF30BD64
:1084A00011F0004F4FEA01314FF4801C4CEA1131BA
:1084B00002D0404261EB410113F0004F4FEA033319
:1084C0004CEA133302D0524263EB430394EA050FA4
:1084D00000F0A780A4F10104D5F1200E0DDB02FA13
:1084E0000EFC22FA05F2801841F1000103FA0EF2A7
:1084F000801843FA05F359410EE0A5F120050EF16D
:10850000200E012A03FA0EFC28BF4CF0020C43FA9D
:1085100005F3C01851EBE37101F0004507D54FF0AA
:10852000000EDCF1000C7EEB00006EEB0101B1F5FA
:10853000801F1BD3B1F5001F0CD349085FEA300040
:108540004FEA3C0C04F101044FEA445212F5800F4B
:1085500080F09A80BCF1004F08BF5FEA500C50F1E8
:10856000000041EB045141EA050130BD5FEA4C0CCB
:10857000404141EB010111F4801FA4F10104E9D154
:1085800091F0000F04BF01460020B1FA81F308BF4B
:108590002033A3F10B03B3F120020CDA0C3208DD17
:1085A00002F1140CC2F10C0201FA0CF021FA02F1F2
:1085B0000CE002F11402D8BFC2F1200C01FA02F162
:1085C00020FA0CFCDCBF41EA0C019040E41AA2BF87
:1085D00001EB0451294330BD6FEA04041F3C1CDA4F
:1085E0000C340EDC04F11404C4F1200220FA04F06F
:1085F00001FA02F340EA030021FA04F345EA030119
:1086000030BDC4F10C04C4F1200220FA02F001FADA
:1086100004F340EA0300294630BD21FA04F029465C
:1086200030BD94F0000F83F4801306BF81F48011F5
:108630000134013D4EE77FEA645C18BF7FEA655C68
:1086400029D094EA050F08BF90EA020F05D054EA3A
:10865000000C04BF1946104630BD91EA030F1EBF3F
:108660000021002030BD5FEA545C05D14000494143
:1086700028BF41F0004130BD14F580043CBF01F536
:10868000801130BD01F0004545F0FE4141F470011C
:108690004FF0000030BD7FEA645C1ABF19461046F7
:1086A0007FEA655C1CBF0B46024650EA013406BFF8
:1086B00052EA033591EA030F41F4002130BD00BFB7
:1086C00090F0000F04BF0021704730B54FF4806474
:1086D00004F132044FF000054FF0000150E700BFF5
:1086E00090F0000F04BF0021704730B54FF4806454
:1086F00004F1320410F0004548BF40424FF0000141
:108700003EE700BF42004FEAE2014FEA31014FEA83
:1087100002701FBF12F07F4393F07F4F81F06051D2
:10872000704792F0000F14BF93F07F4F704730B541
:108730004FF4607401F0004521F0004120E700BFD4
:1087400050EA010208BF704730B54FF000050AE05B
:1087500050EA010208BF704730B511F0004502D55C
:10876000404261EB41014FF4806404F132045FEA5E
:10877000915C3FF4DCAE4FF003025FEADC0C18BF03
:1087800003325FEADC0C18BF033202EBDC02C2F1F9
:10879000200300FA03FC20FA02F001FA03FE40EA8B
:1087A0000E0021FA02F11444C1E600BF4FEA410273
:1087B000B2F1E04324BFB3F5001CDCF1FE5C0DD93F
:1087C00001F0004C4FEAC0024CEA5070B2F1004F89
:1087D00040EB830008BF20F00100704711F0804F8C
:1087E00021D113F13872BCBF01F00040704741F451
:1087F00080114FEA5252C2F11802C2F1200C10FA55
:108800000CF320FA02F018BF40F001004FEAC12338
:108810004FEAD32303FA0CFC40EA0C0023FA02F3DC
:108820004FEA4303CCE77FEA625307D150EA0133B2
:108830001EBF4FF0FE4040F44000704701F0004082
:1088400040F0FE4040F40000704700BF80F0004060
:1088500002E000BF81F0004142001FBF5FEA410318
:1088600092EA030F7FEA226C7FEA236C6AD04FEA18
:108870001262D2EB1363C1BFD2184140484041405D
:10888000B8BF5B42192B88BF704710F0004F40F40F
:10889000000020F07F4018BF404211F0004F41F42B
:1088A000000121F07F4118BF494292EA030F3FD0F7
:1088B000A2F1010241FA03FC10EB0C00C3F120030A
:1088C00001FA03F100F0004302D5494260EB400099
:1088D000B0F5000F13D3B0F1807F06D340084FEA04
:1088E000310102F10102FE2A51D2B1F1004F40EBF9
:1088F000C25008BF20F0010040EA03007047490061
:1089000040EB000010F4000FA2F10102EDD1B0FA2B
:1089100080FCACF1080CB2EB0C0200FA0CF0AABF20
:1089200000EBC25052421843BCBFD04018437047BE
:1089300092F0000F81F4000106BF80F400000132C4
:10894000013BB5E74FEA41037FEA226C18BF7FEA9B
:10895000236C21D092EA030F04D092F0000F08BFDD
:108960000846704790EA010F1CBF0020704712F0C4
:108970007F4F04D1400028BF40F00040704712F103
:1089800000723CBF00F50000704700F0004343F068
:10899000FE4040F4000070477FEA226216BF08469E
:1089A0007FEA23630146420206BF5FEA412390EA61
:1089B000010F40F4800070474FF0000304E000BF57
:1089C00010F0004348BF40425FEA000C08BF704708
:1089D00043F0964301464FF000001CE050EA0102CC
:1089E00008BF70474FF000030AE000BF50EA0102E1
:1089F00008BF704711F0004302D5404261EB4101CE
:108A00005FEA010C02BF84460146002043F0B643F2
:108A100008BFA3F18053A3F50003BCFA8CF2083A17
:108A2000A3EBC25310DB01FA02FC634400FA02FC20
:108A3000C2F12002BCF1004F20FA02F243EB020027
:108A400008BF20F00100704702F1200201FA02FC89
:108A5000C2F1200250EA4C0021FA02F243EB02007C
:108A600008BF20EADC7070474FF0FF0C1CEAD052C0
:108A70001EBF1CEAD15392EA0C0F93EA0C0F6FD081
:108A80001A4480EA010C400218BF5FEA41211ED05F
:108A90004FF0006343EA501043EA5111A0FB01314B
:108AA0000CF00040B1F5000F3EBF490041EAD37120
:108AB0005B0040EA010062F17F02FD2A1DD8B3F19C
:108AC000004F40EBC25008BF20F00100704790F00B
:108AD000000F0CF0004C08BF49024CEA502040EA5D
:108AE00051207F3AC2BFD2F1FF0340EAC250704723
:108AF00040F400004FF00003013A5DDC12F1190F61
:108B0000DCBF00F000407047C2F10002410021FAD2
:108B100002F1C2F1200200FA02FC5FEA310040F1EA
:108B2000000053EA4C0308BF20EADC70704792F063
:108B3000000F00F0004C02BF400010F4000F013A9B
:108B4000F9D040EA0C0093F0000F01F0004C02BF96
:108B5000490011F4000F013BF9D041EA0C018FE705
:108B60000CEAD15392EA0C0F18BF93EA0C0F0AD00B
:108B700030F0004C18BF31F0004CD8D180EA010031
:108B800000F00040704790F0000F17BF90F0004FCA
:108B9000084691F0000F91F0004F14D092EA0C0FAC
:108BA00001D142020FD193EA0C0F03D14B0218BF3F
:108BB000084608D180EA010000F0004040F0FE4085
:108BC00040F40000704740F0FE4040F44000704721
:108BD0004FF0FF0C1CEAD0521EBF1CEAD15392EAA0
:108BE0000C0F93EA0C0F69D0A2EB030280EA010C90
:108BF00049024FEA402037D04FF0805343EA111129
:108C000043EA10130CF000408B4238BF5B0042F186
:108C10007D024FF4000C8B4224BF5B1A40EA0C002B
:108C2000B3EB510F24BFA3EB510340EA5C00B3EB5D
:108C3000910F24BFA3EB910340EA9C00B3EBD10F4B
:108C400024BFA3EBD10340EADC001B0118BF5FEA9D
:108C50001C1CE0D1FD2A3FF650AF8B4240EBC250C6
:108C600008BF20F0010070470CF0004C4CEA502087
:108C70007F32C2BFD2F1FF0340EAC250704740F4D6
:108C800000004FF00003013A37E792F0000F00F0C8
:108C9000004C02BF400010F4000F013AF9D040EA46
:108CA0000C0093F0000F01F0004C02BF490011F4DA
:108CB000000F013BF9D041EA0C0195E70CEAD153D2
:108CC00092EA0C0F08D142027FF47DAF93EA0C0FB9
:108CD0007FF470AF084676E793EA0C0F04D14B029D
:108CE0003FF44CAF08466EE730F0004C18BF31F04F
:108CF000004CCAD130F000427FF45CAF31F0004349
:108D00007FF43CAF5FE700BF4FF0FF3C06E000BFE1
:108D10004FF0010C02E000BF4FF0010C4DF804CD04
:108D20004FEA40024FEA41037FEA226C18BF7FEA14
:108D3000236C11D001B052EA530C18BF90EA010F16
:108D400058BFB2EB030088BFC81738BF6FEAE170A5
:108D500018BF40F0010070477FEA226C02D15FEA41
:108D6000402C05D17FEA236CE4D15FEA412CE1D0AD
:108D70005DF8040B704700BF844608466146FFE774
:108D80000FB5FFF7C9FF002848BF10F1000F0FBD56
:108D90004DF808EDFFF7F4FF0CBF012000205DF84F
:108DA00008FB00BF4DF808EDFFF7EAFF34BF0120D4
:108DB00000205DF808FB00BF4DF808EDFFF7E0FF6D
:108DC00094BF012000205DF808FB00BF4DF808EDBE
:108DD000FFF7D2FF94BF012000205DF808FB00BF21
:108DE0004DF808EDFFF7C8FF34BF012000205DF803
:108DF00008FB00BF4FEA40024FEA41037FEA226CC2
:108E000002D15FEA402C08D17FEA236C02D15FEAED
:108E1000412C02D14FF0000070474FF00100704725
:108E2000014B1868704700BF0802002070B50F4E54
:108E30000F4D761BB61018BF002405D0013455F82D
:108E4000043B9847A642F9D10A4E0B4D761B03F01E
:108E5000A9FAB61018BF002406D0013455F8043B17
:108E60009847A642F9D170BD70BD00BFB0C34000A5
:108E7000B0C34000B8C34000B0C340000FB400B559
:108E8000074983B004AB086853F8042B8168019349
:108E900000F024FE03B05DF804EB04B0704700BF9F
:108EA00008020020024B0146186800F00BB800BF12
:108EB00008020020024B0146186801F02BBF00BFDA
:108EC000080200202DE9F04F01F10B06162E83B0A9
:108ED000054640F29E8036F0070600F1BD80B142A3
:108EE00000F2BA8000F040FCB6F5FC7FC0F093823F
:108EF000730A00F0B880042B00F27981B30903F102
:108F0000390003F1380EC300BF4F3B44A3F1080101
:108F10005C68A14206D10CE0002A80F2AA80E468D5
:108F2000A14206D0636823F003039A1B0F2AF3DDE6
:108F300070463C69DFF8E4E2744500F0AB81636899
:108F400023F003039A1B0F2A00F39081002AC7F82D
:108F500014E0C7F810E080F29D80B3F5007F80F048
:108F60006181DB0803F1010C99107A6857F83C80A5
:108F7000C4F8088001238B4007EBCC011343083968
:108F8000E1607B6047F83C40C8F80C408210012447
:108F900094409C4200F28B801C4206D120F00300DA
:108FA00064001C4200F10400FAD007EBC009CC4673
:108FB0008046DCF80C309C4507D16DE1002A80F238
:108FC0007B81DB689C4500F06781596821F00301D3
:108FD0008A1B0F2AF2DDD3F80CC0D3F80880009367
:108FE0009C19284646F0010642F001055E60C8F86B
:108FF0000CC0CCF808807C613C61C4F80CE0C4F87B
:1090000008E065605A5000F0B5FB009B03F10804CE
:109010001EE0102920D800F0A7FB102618230220FC
:10902000794F3B44A3F108025C68944200F03D8113
:109030006368E168A66823F00303234428465A685E
:10904000F16042F001028E605A6000F093FB083438
:10905000204603B0BDE8F08F00240C2320462B608F
:1090600003B0BDE8F08F40204FF400734FF03F0E87
:109070004AE72344E1685A68A66842F00102F160B9
:1090800028468E605A6000F075FB0834204603B015
:10909000BDE8F08F234428465A6842F001025A6026
:1090A00000F068FB0834204603B0BDE8F08FBC68D0
:1090B000636823F00308B04504D3A8EB06030F2B25
:1090C00000F38580DFF85891504BD9F800201B68D9
:1090D0000132334404EB080A00F0558103F5805354
:1090E0000F3323F47F6B2BF00F0B5946284600F00B
:1090F00047FB411C024600F0FC80824500F2F780ED
:10910000434B19685944196000F04D81D9F80000AB
:1091100001301BBFA2EB0A0A5144C9F800201960B4
:1091200012F0070100F01581C1F10800C1F580516E
:109130000244083102EB0B09C9F30B09A1EB090941
:10914000494628460193009200F01AFB431C9DE813
:109150000C0000F04381801A484440F00100196877
:10916000BA604944BC425060196017D0B8F10F0F83
:1091700040F2FB806068A8F10C0222F0070204EBC9
:10918000020E00F001004FF0050C10430F2A606042
:10919000CEF804C0CEF808C000F217811D4BBC68A1
:1091A0001A68914288BF19601B4B1A689142626825
:1091B00088BF196022F003029642A2EB060301D891
:1091C0000F2B04DC284600F0D5FA002440E7A21952
:1091D00043F0010346F0010666602846BA6053601A
:1091E00000F0C8FA0834204603B0BDE8F08F142B15
:1091F00071D9542B00F2A380330B03F16F0003F1FC
:109200006E0EC30080E600BF38060020C00E0020AE
:10921000900E0020B80E0020BC0E0020400600205A
:10922000400A00205A0A042A5BD9142A00F2AE80B0
:1092300002F15C01C9005B3207EB010C7958ACF11B
:10924000080C8C4500F088804A6822F003029342A3
:1092500073D289688C45F7D1DCF80C207B68E2601A
:10926000C4F808C09460CCF80C408FE6A11946F011
:10927000010C42F00106C4F804C028467961396146
:10928000C1F80CE0C1F808E04E60E25000F072FA5C
:109290000834DDE67B6879E608F1010818F0030F71
:1092A0000CF1080C7FF485AE2DE0DC68A34208BF0A
:1092B00002303FF43EAEBBE619441C464A68DB6808
:1092C00054F8086F42F001024A602846F3609E603D
:1092D00000F050FABCE603F15C0003F15B0EC30042
:1092E00012E69A0902F13901C9003832A4E7BC42FA
:1092F00054D0BC68626822F003025DE759F808396F
:10930000994540F0868010F0030F00F1FF30F5D151
:109310007B6823EA04037B6064009C423FF6C7AE8F
:10932000002C3FF4C4AE1C4240467FF43EAE6400C5
:109330001C4200F10400FAD037E68C468CE7B3F506
:10934000AA7F15D8F30B03F1780003F1770EC30061
:10935000DAE54FF48051EDE67B689210012101FAC5
:1093600002F213437B60624679E70123536029E7E9
:1093700040F25452934222D8B30C03F17D0003F122
:109380007C0EC300C0E503F1100BAEE6542A29D8C9
:109390001A0B02F16F01C9006E324DE7204B1968BC
:1093A00059441960B2E6CAF30B0000287FF4AEAE50
:1093B00008EB0B03BA6843F001035360EEE67F202D
:1093C0004FF47E734FF07E0E9EE504F108012846AF
:1093D000009301F09FFC009B1968DFE601204FF02D
:1093E0000009BCE6B2F5AA7F05D8DA0B02F17801D4
:1093F000C900773220E740F254518A4205D89A0CCE
:1094000002F17D01C9007C3216E74FF47E717E22A5
:1094100012E77B6880E7F00806F1080300E600BF6A
:10942000900E00200000000000000000000000007E
:1094300001F0FF01102A2BDB10F0070F08D010F805
:10944000013B013A8B422DD010F0070F42B3F6D109
:10945000F0B441EA012141EA014122F007047FF022
:1094600000070023F0E80256083C85EA010586EA79
:10947000010685FA47F5A3FA87F586FA47F6A5FAB5
:1094800087F68EB9EED1F0BC01F0FF0102F00702C1
:1094900032B110F8013B013A83EA010313B1F8D16C
:1094A0000020704701387047002D06BF354603384D
:1094B000073815F0010F07D1013015F4807F02BF86
:1094C000013015F4C03F0130F0BC0138704700BFD7
:1094D000844641EA000313F003036DD1403A41D3BF
:1094E00051F8043B40F8043B51F8043B40F8043B7E
:1094F00051F8043B40F8043B51F8043B40F8043B6E
:1095000051F8043B40F8043B51F8043B40F8043B5D
:1095100051F8043B40F8043B51F8043B40F8043B4D
:1095200051F8043B40F8043B51F8043B40F8043B3D
:1095300051F8043B40F8043B51F8043B40F8043B2D
:1095400051F8043B40F8043B51F8043B40F8043B1D
:1095500051F8043B40F8043B51F8043B40F8043B0D
:10956000403ABDD2303211D351F8043B40F8043BAD
:1095700051F8043B40F8043B51F8043B40F8043BED
:1095800051F8043B40F8043B103AEDD20C3205D3BD
:1095900051F8043B40F8043B043AF9D2043208D0B5
:1095A000D2071CBF11F8013B00F8013B01D30B8827
:1095B00003806046704700BF082A13D38B078DD005
:1095C00010F003038AD0C3F10403D21ADB071CBFD7
:1095D00011F8013B00F8013B80D331F8023B20F841
:1095E000023B7BE7043AD9D3013A11F8013B00F87A
:1095F000013BF9D20B7803704B7843708B78837002
:10960000604670478842F0B50DD98B1898420AD24F
:109610008418002A51D0224613F8014D02F8014D5A
:109620009942F9D1F0BD0F2A48D941EA00039B07BE
:1096300046D100F1100401F11003154653F8106CE7
:1096400044F8106C53F80C6C44F80C6C53F8086C2C
:1096500044F8086C103D53F8046C44F8046C0F2D6A
:1096600003F1100304F11004E8D8A2F1100323F071
:109670000F0302F00F0E1033BEF1030F1944034421
:1096800021D91E1F0D467446043C55F8047B46F84C
:10969000047F032CF8D8AEF1040424F0030404344E
:1096A0002144234402F0030262B1013B0A4411F851
:1096B000014B03F8014F8A42F9D1F0BD0346F3E7AD
:1096C0000346F2E7F0BD7246EEE700BF70B48607CE
:1096D00046D0541E002A41D0CAB2034602E014F11B
:1096E000FF343BD303F8012B9D07F8D1032C2ED96F
:1096F000CDB245EA05250F2C45EA054519D903F1F8
:1097000010022646103E0F2E42F8105C42F80C5C08
:1097100042F8085C42F8045C02F11002F2D8A4F1AD
:10972000100222F00F0204F00F041032032C134435
:109730000DD91E462246043A032A46F8045BFAD89D
:10974000221F22F003020432134404F003042CB15C
:10975000C9B21C4403F8011B9C42FBD170BC70478A
:1097600014460346C2E700BF014801F06DBD00BFCB
:109770009C1B0020014801F069BD00BF9C1B00201C
:1097800038B5074C0023054608462360FCF782FFE6
:10979000431C00D038BD2368002BFBD02B6038BDA4
:1097A000B01B002000290CBF022200224FF480636E
:1097B00000F000B82DE9F043614C256883B0044601
:1097C0000F4690461E4615B1AB6B002B64D0B8F126
:1097D000020F06D0B8F1010F00F29F80002EC0F2F8
:1097E0009C80636ED80734D52146284601F014F9D1
:1097F000216B41B104F14003994202D0284601F0A7
:1098000089FA00232363B4F90C300022A26162605C
:109810001A063AD423F44A6323F00303B8F1020F83
:10982000A3811DD001AB6A462146284601F010FDF8
:10983000A3891843A081002E32D1009E3046FFF745
:1098400031FB074600286BD0A38943F08003A38136
:1098500028E0A3899905C7D4A06D01F0F5FCC3E702
:109860000025616E002604F1430243F0020301204B
:10987000A660CE07A38122602261606101D49805B1
:109880003ED5284603B0BDE8F0832169284601F0A3
:1098900041FAB4F90C30BDE7284601F015F996E716
:1098A000002FCBD0AB6B002B33D0009BB4F90C2036
:1098B00027609E421CBF42F40062A281B8F1010FF2
:1098C00004BF42F00102A28192B212F008032761A4
:1098D00066610ED0D1071AD5656E7642002315F069
:1098E0000105A661A36009D00025284603B0BDE8A4
:1098F000F083A360656E15F00105F5D19305C0D422
:10990000A06D01F0A3FC284603B0BDE8F083A6607B
:10991000F0E7284601F0D8F8C7E74FF0FF35B0E789
:10992000DDF80090B14504D04846FFF7BBFA074682
:1099300020B9B4F90C304FF0FF3592E74E4683E77B
:1099400008020020000000000000000000000000ED
:109950000000000000000000000000000000000007
:1099600000000000000000000000000000000000F7
:1099700000000000000000000000000000000000E7
:1099800090F800F06DE9024520F007016FF0000C3F
:1099900010F0070491F820F040F049804FF00004E7
:1099A0006FF00700D1E9002391F840F000F10800C2
:1099B00082FA4CF2A4FA8CF283FA4CF3A2FA8CF3FA
:1099C0004BBBD1E9022382FA4CF200F10800A4FA61
:1099D0008CF283FA4CF3A2FA8CF3E3B9D1E90423B5
:1099E00082FA4CF200F10800A4FA8CF283FA4CF3EC
:1099F000A2FA8CF37BB9D1E9062301F1200182FAA6
:109A00004CF200F10800A4FA8CF283FA4CF3A2FAAB
:109A10008CF3002BC6D0002A04BF04301A4612BAB9
:109A2000B2FA82F2FDE8024500EBD2007047D1E9BC
:109A3000002304F00305C4F100004FEAC50514F04B
:109A4000040F91F840F00CFA05F562EA05021CBF1C
:109A500063EA050362464FF00004A9E72DE9F84FD9
:109A60004B6E9C0493462FD59368126853B30E46F1
:109A7000074602F1080919E920045FEA9A0817D09D
:109A8000043D002401E0A04510D0324655F8041FE3
:109A9000384601F0BBF8431C04F10104F3D1002364
:109AA000CBF80830CBF80430BDE8F88FDBF808308D
:109AB0002AF0030AA3EB0A03CBF8083009F10809DE
:109AC000002BD8D10020EAE701F00AFA0023CBF8F6
:109AD0000830CBF80430BDE8F88F00BF2DE9F04F17
:109AE000ADB01D468B4690460793069018B1836B28
:109AF000002B00F0F380DBF86430BBF90C00DF07CB
:109B000081B202D48E0540F1FC808C040AD4DBF8CB
:109B1000643040F4005123F40053ABF80C10CBF840
:109B2000643089B2080740F1B380DBF81030002BB5
:109B300000F0AE8001F01A030A2B00F0B58000237C
:109B40000DF170090B93119310930393CDF83C9092
:109B5000CA46CDF810B098F800304446FBB1252B2A
:109B600002D11CE0252B03D014F8013F002BF9D1C2
:109B7000A4EB08059DB1109B119ACAF8008001332F
:109B80002A44072BCAF80450119210937ADD002A58
:109B900040F0B084039B10922B44CA460393237871
:109BA000002B00F0E08300204FF000038DF83730E9
:109BB00004F1010862780546064603464FF0FF347B
:109BC00008F10108A2F12001582900F2DE82DFE845
:109BD00011F02102DC02DC022902DC02DC02DC02E0
:109BE000DC02DC02DC0289029502DC02A200BD027A
:109BF000DC029F01A401A401A401A401A401A40109
:109C0000A401A401A401DC02DC02DC02DC02DC020F
:109C1000DC02DC02DC02DC02DC02B201DC02DC027F
:109C2000DC02DC02DC02DC02DC02DC02DC02DC0244
:109C30009701DC02DC02DC02DC02DC029B01DC02BC
:109C4000DC025302DC02DC02DC02DC02DC02DC02AD
:109C5000DC02DC02DC02DC025A021B02DC02DC0257
:109C6000DC026E021B02DC02DC027302DC02F50184
:109C700082010902D702DC029A02DC02A700DC02A0
:109C8000DC022E020AF1080A039B2B44039386E7A9
:109C90005946069800F0ACFD18BBBBF80C1001F05B
:109CA0001A030A2B7FF44BAFBBF90E30002BFFF6E3
:109CB00046AFDBF86430DB0705D48F0503D4DBF84F
:109CC000580001F0C3FA2B4642465946069800F068
:109CD0004DFD039003982DB0BDE8F08F00F0F4FE29
:109CE00009E7DBF86430D90704D4BBF80C309A05D7
:109CF00040F1AA844FF0FF33039303982DB0BDE8E1
:109D0000F08FDBF8580001F09FFABBF90C0081B22C
:109D1000FBE67642079243F0040398F800204FE7F1
:109D200008969E0600F150840799DD060A4600F168
:109D3000EF83580640F1EC830E880431002701229E
:109D400007914FF000018DF837100025611C00F0DD
:109D5000168123F08001029156EA070140F0148138
:109D6000002C40F05C83002A40F0B78313F001031D
:109D7000059300F057840DF1B00B30230BF8413DF3
:109D8000059BA342B8BF234601930DB10133019354
:109D9000029B13F00203099302D0019B023301934B
:109DA000029B13F084030A9340F01782089B019AE8
:109DB0009D1A002D40F31182102D40F39084109BCA
:109DC000119AC44ED6461027A2461946069C07E0B3
:109DD00001F1020C0EF1080E0146103D102D11DDAF
:109DE000481C1032072811928EE8C0001090EFDD59
:109DF000002A40F0E481103D102D11464FF0010C77
:109E0000CE46EDDC54466146F2462A4407291192BB
:109E1000CAF80060CAF80450109100F3EC829DF873
:109E200037500AF1080A481C002D40F0DE81099BDA
:109E3000002B00F0F88102320EA9022307281192AC
:109E400010908AE80A0040F3EA81002A40F08C83EF
:109E50000A9B802B4FF001001146CA4640F0E78173
:109E6000089B019D5E1B002E40F3E181102E9A4D50
:109E700040F35084D4461027A246069C07E001F127
:109E8000020E0CF1080C0146103E102E11DD481C8C
:109E90001032072811928CE8A0001090EFDD002A04
:109EA00040F09D82103E102E4FF0010E1146CC4620
:109EB000EDDC5446E2463244BEF1070F11928AE8C7
:109EC0006000CDF840E000F369830AF1080A0EF162
:109ED00001007146ABE1089613F0200240F08C833C
:109EE00013F0100140F01A8313F0400200F01683C3
:109EF00007980A460146043106880791002720E7A3
:109F0000089643F01003E7E7089643F0100308E7CC
:109F100043F0800398F8002052E6A2F130010026B9
:109F200018F8012B06EB860601EB4606A2F130017C
:109F30000929F5D946E60896002840F0088443F040
:109F400010039E0600F14C83DD0600F1F3825806F3
:109F500040F1F082079DB5F900602A46F7170432F8
:109F6000304639460792002871F10002C0F25D8345
:109F7000611C9DF837504FF001027FF4EAAE56EABB
:109F8000070100F04D820293012A00F08C82022A20
:109F900040F05C820B98CB46330906F00F0143EA90
:109FA00007733A091E461746435C0BF8013D56EA13
:109FB0000703F1D1A9EB0B030593E1E6002840F07C
:109FC000C083990600F16783DA0600F1F1805B0631
:109FD00040F1EE80079A136804320792BDF80C2016
:109FE0001A80B8E507983D4A08960B9206687822D1
:109FF000302104308DF8392043F002030790002708
:10A000008DF8381002229CE60896002899D08DF829
:10A01000375096E798F80020002D7FF4D1AD01204D
:10A020002025CDE543F0010398F80020C8E5089607
:10A03000002840F0938329490B919F0600F1E882A4
:10A040000798DE06014600F170825D0640F16D82E0
:10A050000431068807910027D80740F1228256EA8A
:10A06000070100F01E8230218DF8392043F00203F1
:10A070008DF83810022264E60896002840F06B83C1
:10A0800017490B91D9E7079908960A688DF8482077
:10A090004FF000000A468DF837000432012001908D
:10A0A000079205900DF1480B0293002470E643F0EF
:10A0B000400398F8002083E598F800206C2A03BF3D
:10A0C00098F8012043F0200308F1010843F0100341
:10A0D00076E500BF70C2400080C2400054C240001C
:10A0E00040C2400007990E680A46002E02F10402A1
:10A0F000FFF60FAE079298F8002061E598F800206F
:10A1000001202B255CE507990896D1F800B04FF0A7
:10A1100000028DF837200E1DBBF1000F00F0E58224
:10A12000671C00F0C4822246002158460193FFF7C5
:10A130007FF9019B002800F0E582A0EB0B0205925D
:10A14000079602939DF83750002419E698F80020EE
:10A150002A2A08F1010700F0E982A2F13001092959
:10A16000B8464FF000043FF62DAD18F8012B04EB74
:10A17000840401EB4404A2F130010929F5D921E559
:10A1800043F0200398F800201AE50896002840F0D4
:10A19000DB82002A00F0E78001218DF848204FF093
:10A1A000000201918DF8372005910DF1480B7BE7F6
:10A1B000079A136804320792039A1A60CBE40FAA35
:10A1C00004992046FFF74AFC002840F03981109995
:10A1D000119A01F1010CCE46FFE51099119A481C25
:10A1E0009DF83750002D3FF422AE01320DF13705B6
:10A1F0000121072811921090CAF80050CAF80410E3
:10A2000040F30881002A40F0BC81099B002B3FF4F9
:10A210001FAE0EAB022208461C931D92CA46014691
:10A220000AF1080A01300A9B802B3FF419AE059B06
:10A23000E41A002C2EDD102CB34D1EDDD646102660
:10A24000069FDDF810A006E0881C0EF1080E1946E6
:10A25000103C102C10DD4B1C1032072B11928EE895
:10A2600060001093F0DD002A65D1103C102C4FF0F7
:10A2700001001146CE46EEDCF24622440728119238
:10A28000CAF80050CAF80440109000F385800AF123
:10A29000080A01300599CAF800B00A44072811924B
:10A2A000CAF80410109040F38280002A40F0188110
:10A2B000029B1092580735D5089B01995C1A002C17
:10A2C00040F3E780CA46102C40F3188210998F4E55
:10A2D000069FDDF810B0102506E0881C0AF1080A78
:10A2E0001946103C102C11DD4B1C1032072B11921B
:10A2F000CAF80060CAF804501093EEDD42BB103C6F
:10A30000102C4FF001001146CA46EDDC224407280C
:10A310001192CAF80060CAF80440109051DD002A7A
:10A3200040F09B81039B089A01998A42ACBF9B181D
:10A330005B1803934EE00FAA51463846FFF78EFB99
:10A34000002840F03F811099119A481CCE467FE7C3
:10A350000FAA59463846FFF781FB60B91099119A48
:10A36000481CCA46BDE7119BDDF810B0002B40F039
:10A37000D48100231093DBF8643013F0010FBBF895
:10A380000C3002D19A0540F1DE805B063FF5B2AC9D
:10A3900003982DB0BDE8F08F002A40F00681059AA1
:10A3A0001D9201231192CDF870B01093CA460AF1A4
:10A3B000080A029B590704D5089B01995C1A002CD6
:10A3C00081DC039B089901988142ACBF5B181B1884
:10A3D000039372BB00231093CA46FFF7BCBB0FAABE
:10A3E00004992046FFF73AFB50BB1099119A01F1EE
:10A3F000010ECC4648E5002A40F040819DF8371018
:10A40000002900F01B8101220DF1370110461D9239
:10A410001C91CA4601460AF1080A013007E5029B71
:10A42000012A00F09880022A0DD10293002600270D
:10A43000B0E50FAA04990698FFF710FB0028C9D0D1
:10A44000DDF810B097E7029300260027494600E0A8
:10A450005946F20842EA4772F80806F00703074631
:10A460001646303356EA070201F8013C01F1FF3B82
:10A47000EED1029AD6077FF59DAD302B3FF49AAD11
:10A48000023930230BF8013CA9EB010305938B46FD
:10A4900076E4039B089A8A42ACBF9B185B1803932F
:10A4A00098E702224DE4002F08BF0A2E52D3CB4674
:10A4B000304639460A22002301F010FB30320BF8F7
:10A4C000012D3046394600230A2201F007FB0646DB
:10A4D0000F4656EA0703EBD16CE50594CB464FE4F3
:10A4E0000FAA04990698FFF7B9FA0028A8D1119A83
:10A4F000CA465EE70FAA04990698FFF7AFFA00284C
:10A500009ED1CA46FFF7C0BB80C2400070C2400067
:10A510000431166807910122002712E407980146CA
:10A5200004310668079100270BE40E680431079197
:10A53000002791E507990E680A46F717043207923B
:10A54000304639460FE5DBF8580000F07FFEBBF8D7
:10A550000C301AE7029B02930DF1B00B3036012349
:10A560000BF8416D05930BE40FAA04990698FFF7C9
:10A5700075FA00287FF464AF1099119A481CCA46F6
:10A5800051E60FAA04990698FFF768FA00287FF4AD
:10A5900057AF1099119A481CCA4648E4002A40F067
:10A5A000918001201146CA4641E60FAA04990698F7
:10A5B000FFF754FA00287FF443AF1098119A013046
:10A5C000CA4667E6D346D6E6079E073626F0070258
:10A5D00002F10801D2E9006707910122FFF7B1BB40
:10A5E000079E073626F00706D6E9000106F10802A5
:10A5F000079206460F46B6E4079E073626F0070286
:10A6000002F10801D2E9006707910022FFF799BB28
:10A61000079E073626F0070101F108000790D1E9EF
:10A62000006719E5CB46FFF7ABBB2D25764267EBFC
:10A6300047078DF837500122FFF788BB099BB3B954
:10A6400011460120CA46F2E5DBF8580000F0FEFD95
:10A650004FF0FF330393FFF750BB0FAA04990698FE
:10A66000FFF7FCF900287FF4EBAE119AA9E60EABD8
:10A6700002221C931D920120CA46D0E50FAA04991C
:10A680000698FFF7EBF900287FF4DAAE1099119ADB
:10A69000481CCA46A4E5079A03991368CD170846D3
:10A6A000043229460792C3E90001FFF754BA58461D
:10A6B00007960293FFF764F9002405909DF8375040
:10A6C000FFF75EBB0FAA04990698FFF7C7F90028A9
:10A6D0007FF4B6AE1099119A481CCA46A7E51099A6
:10A6E000119A204E0131FFF790BB062C28BF06249B
:10A6F000059407960194DFF870B0D5E41098194ED0
:10A70000013003E605949DF83750079602930446FE
:10A71000FFF736BB8646FFF7CEBB06980FAA594611
:10A72000FFF79CF900283FF424AE24E6079998F837
:10A7300001200C68043144EAE474B8460791FFF73D
:10A740003FBA8DF837503CE48DF8375021E58DF84D
:10A750003750FFF7F4BB8DF8375091E48DF8375040
:10A7600069E400BF70C2400068C240002DE9F041BA
:10A770000C46ADF58D6D8989666EE589199621F0D7
:10A7800002010646E069ADF80C1017464FF48061EF
:10A79000626AADF80E5098461AAD0023079016A8CD
:10A7A00009920693009504950291059100F048FDE9
:10A7B00043463A4669463046FFF790F9051E07DBE7
:10A7C0003046694600F028F9002818BF4FF0FF35E1
:10A7D000BDF80C305B0603D5A38943F04003A38189
:10A7E000169800F02FFD28460DF58D6DBDE8F0811F
:10A7F00038B5304B1B6805460C4613B19A6B002ADE
:10A8000038D0B4F90C2093B218070CD52069A8B140
:10A8100013F001021ED0636900225B42A361A260B3
:10A82000F0B1002038BDD9063CD5580726D42069A0
:10A8300042F00803A3819BB20028E9D103F42072FF
:10A84000B2F5007FE4D02846214600F02FFDA38911
:10A850002069DDE7990758BF6269A2600028E0D14E
:10A86000B4F90C301A06DDD543F04003A3814FF054
:10A87000FF3038BD184600F027F9C2E7216B51B10F
:10A8800004F14003994204D0284600F043FAB4F999
:10A890000C200023236300232069636022F024023C
:10A8A0002060C5E742F0400209232B604FF0FF30E3
:10A8B000A28138BD08020020024B13B1024800F00B
:10A8C00005B870470000000039AB40000023014686
:10A8D0001A46184600F0DABFB1F90C309AB22DE9E9
:10A8E000F0410D46110780463AD46A6843F400638C
:10A8F000002AAB816FDDAC6A002C49D000229BB2EC
:10A90000D8F80060C8F8002013F4805267D02A6D90
:10A910005F0705D569682B6B521A0BB1EB6BD21A26
:10A920000023E9694046A047441C3CD0B5F90C30EF
:10A930002A692A6023F400630022AB81DB046A6089
:10A9400047D4296BC8F8006011B305F14003994260
:10A9500002D0404600F0DEF900202863BDE8F08117
:10A960002E69AEB12C682E6091070CBF6B69002375
:10A97000A41BAB600AE0234632466F6AE969404691
:10A98000B8470028A4EB0004064404DD002CF2DCE8
:10A990000020BDE8F081AB8943F04003AB814FF06C
:10A9A000FF30BDE8F081D8F800401D2CF3D8194BDA
:10A9B000E340DB4313F00103EDD1B5F90C206B60EC
:10A9C00022F400632969AB81DA042960B9D5002C2F
:10A9D000B7D12865B5E7EA6B002A8CDCD8E70123FC
:10A9E000E9694046A047431C024602D0AB89AC6AE5
:10A9F0008EE7D8F80030002BF8D01D2B01D0162B95
:10AA000002D1C8F80060C3E7AB8943F04003AB81D3
:10AA1000BDE8F0810100402038B50D46044608B17C
:10AA2000836BBBB1B5F90C0088B16B6EDB0701D449
:10AA3000810517D520462946FFF74EFF6B6EDA07D2
:10AA4000044602D4AB899B0507D5204638BD044691
:10AA5000204638BD00F038F8E4E7A86D00F0F6FBBA
:10AA6000204638BDA86D00F0EFFBE3E7014900F098
:10AA7000AFBB00BF75B9400010B50023044681810B
:10AA8000C281036043608360436603614361836105
:10AA9000194608225C30FEF719FE07480749084AA4
:10AAA000084B2062E4616162A262E36204F1580033
:10AAB000BDE8104000F0C4BBB9B64000DDB64000B0
:10AAC00019B7400039B7400010B50446124800F0ED
:10AAD000BBFBA26BD2B904F53B731048C4F8E83253
:10AAE0000321C4F8E022E063C4F8E41260680421A2
:10AAF000FFF7C2FF01220921A068FFF7BDFF022274
:10AB00001221E068FFF7B8FF0123A3630248BDE804
:10AB1000104000F09BBB00BF981B00206DAA4000B6
:10AB2000014800F091BB00BFAC1B0020014800F0C1
:10AB30008DBB00BFAC1B002038B50A4C0A4D641B0E
:10AB4000A4100AD004F18043013B05EB8305013CCE
:10AB500055F804399847002CF9D1BDE8384001F088
:10AB60002BBC00BFC8C34000C4C340002DE9F04760
:10AB700082B080468946144600F054FB012836D046
:10AB80004A4604F15C0301A9404600F031FE421C34
:10AB9000064625D0A8B39DF804E000250DF1040A6F
:10ABA00009E023685A1C226083F800E00135B542B1
:10ABB00027D215F80AE0A368013B002BA360F0DA66
:10ABC000A769BB4271462246404602DBBEF10A0F2E
:10ABD000E7D100F0B5FD431CE8D102B0BDE8F08735
:10ABE000A38943F04003A38102B0BDE8F08709F1D7
:10ABF000FF33FE2BC4D85FFA89FE06468DF804E0C9
:10AC0000CBE7484602B0BDE8F08700BF30B5536ED1
:10AC100013F0010FB2F90C30144683B005469AB216
:10AC200001D190051CD5900406D4626E43F4005304
:10AC300042F40052A381626628462246FFF796FF3F
:10AC4000636EDA07054602D4A3899B0502D5284620
:10AC500003B030BDA06D00F0F9FA284603B030BD56
:10AC6000A06D019100F0F0FAB4F90C3001999AB29C
:10AC7000D9E700BFF8B5244F0C460646FEF774FD31
:10AC8000BB685D68C4F57E610F3125F0030529447A
:10AC900021F47F6121F00F01A1F58054B4F5805FAC
:10ACA00007DB00213046FEF76BFDBB682B44984262
:10ACB00004D03046FEF75EFD0020F8BD614230460C
:10ACC000FEF75EFD01300DD0104BBA6819682D1BE0
:10ACD00045F001053046091B55601960FEF74AFD35
:10ACE0000120F8BD00213046FEF74AFDBA68831AFC
:10ACF0000F2BDEDD064C0549246843F00103001BE1
:10AD000053600860D5E700BF38060020900E002091
:10AD1000400A0020002944D02DE9F0410D4680462C
:10AD2000FEF722FD55F8047C694927F00103A5F1DF
:10AD30000804E2188E685068B24220F003005ED02A
:10AD4000FE0750600BD455F8087CE41B01F1080E97
:10AD5000A56875453B446DD0E768EF60BD60151888
:10AD60006D68ED073ED543F001026260E350B3F534
:10AD7000007F17D2DB08581C9A104D6851F83070CC
:10AD8000A7600123934001EBC0022B43083AE26025
:10AD90004B6041F83040FC604046BDE8F041FEF7B2
:10ADA000E9BC70475A0A042A52D89A0902F13907B5
:10ADB000FF0002F13805C819CA59083890424FD02F
:10ADC000516821F003018B4232D292689042F7D150
:10ADD000C368A060E3609C60C4604046BDE8F04189
:10ADE000FEF7C8BC95683B4FBD42034440D0D068D5
:10ADF000E86043F0010285606260E350B7E7FF0757
:10AE0000034407D455F8082CA41A1344A068E26838
:10AE1000C2609060304A126843F001009342606063
:10AE20008C60B9D32D4B40461968FFF723FFB3E779
:10AE30001046CDE711184968C90744D49168D26813
:10AE4000CA60034443F0010091606060E350A3E7EF
:10AE5000142A16D802F15C07FF0002F15B05AAE78D
:10AE6000AA1001234D6893402B434B600346B0E783
:10AE700043F001024C610C61E560A5606260E35043
:10AE80008AE7542A06D81A0B02F16F07FF0002F175
:10AE90006E0590E7B2F5AA7F06D8DA0B02F17807C3
:10AEA000FF0002F1770586E740F25450824206D84F
:10AEB0009A0C02F17D07FF0002F17C057BE74FF45D
:10AEC0007E777E2577E743F001016160136063E7D9
:10AED0003806002040060020440A0020C00E002052
:10AEE0009368002B73D02DE9F04F8B8983B00C460B
:10AEF00019070090164626D5226922B313F00200E6
:10AF000035682CD04FF00009B04FC846B246B8455E
:10AF100043464A4628BF3B460098B8F1000F50D040
:10AF2000E169666AB047002858DDDAF808301B1A74
:10AF30008144A8EB0008CAF80830002BE7D10020B4
:10AF400003B0BDE8F08F21460098FFF751FC0028C0
:10AF500040F03381A389356813F00200D2D113F099
:10AF6000010945D14F46019637B39A05D4F80880B8
:10AF700040F183804745C346C0F0AB8013F4906F27
:10AF800040F0AC802068BA465A464946FEF73AFB84
:10AF9000A2682368A2EB08025B44A2602360019AC6
:10AFA0009368A3EB0A03D144A7EB0A079360002B35
:10AFB000C5D0A389002FD8D1D5F800906F68083587
:10AFC000D2E7D5F80090D5F8048008359FE7002037
:10AFD000704721460098FFF71FFD70B3B4F90C309D
:10AFE00043F040034FF0FF30A38103B0BDE8F08F82
:10AFF000814633464E46A8469A464D464EB380B3E8
:10B00000206823696269B145CB4628BFB3469842A0
:10B010005F4604D9A36813449B4500F3A68093457B
:10B020004BDB1346676AE16900982A46B847071E5A
:10B03000D4DDB9EB0709CCD00120DAF80830DB1BEE
:10B040003D44F61BCAF80830002B3FF478AF002EC1
:10B05000D5D108F1080313E9600098460833002EA3
:10B06000F9D032460A212846FEF7E2F9002800F01E
:10B07000A1800130A0EB0509C2E72068236998424E
:10B0800002D863699F425DD2B84528BFB8464246A0
:10B090004946FEF7B7FAA3682268A3EB08034244C7
:10B0A000A36022600BB1C24679E721460098FFF702
:10B0B000B3FC002892D1C24671E75A462946FEF7F2
:10B0C000A1FAA2682368A2EB0B025B44A260236092
:10B0D000AFE72068B846BA46BB4655E762692068C4
:10B0E000216902EB4208A0EB010A08EBD8780AF1CB
:10B0F00001004FEA680838444045424684BF804614
:10B1000042465B0544D511460098FDF7DBFE8346B9
:10B11000002855D052462169FEF7DAF9A38923F4B5
:10B12000906343F08003A3810BEB0A00A8EB0A03B2
:10B13000C4F810B0C4F814802060A360B846BA46C2
:10B14000BB4621E76FF00041B94228BF39464A4665
:10B1500091FBF3F10098666A03FB01F3E169B047E4
:10B16000B0F1000A3FF71BAF38E71A4629460193B2
:10B17000FEF748FA2268019B00981A442260214693
:10B18000FFF74AFC019B00287FF428AF1F4650E7D9
:10B19000009800F0EBF883460028C5D1009D216996
:10B1A0002846FFF7B7FDB4F90C300C2223F08003DA
:10B1B0002A6015E706F1010922E74FF0FF30BFE6EC
:10B1C000009A0C231360B4F90C3009E700FCFF7FF0
:10B1D0002DE9F84310F538771FD0884606464FF022
:10B1E00000097D68BC68013D11D4A389012B05F1DC
:10B1F000FF3508D9B4F90E3001332146304602D06C
:10B20000C04749EA00096B1C04F16804EDD13F68AE
:10B21000002FE6D14846BDE8F883B9464846BDE868
:10B22000F88300BF044B054A1B685B6B002B08BF0B
:10B23000134693F828017047080200204C0A0020AA
:10B24000704700BF704700BF704700BF704700BF26
:10B2500070B50C46B1F90E10002990B015461E4687
:10B2600014DB01AA00F0E8FB00280FDB029A02F4CD
:10B270007042A2F50052B2FA82F252094FF4806392
:10B280004FF4006032602B6010B070BDA2890023C3
:10B2900012F08000336004D0402218462A6010B0BB
:10B2A00070BD4FF480632B6010B070BD8A89920727
:10B2B0000B4606D501F1430201211A601A6159615A
:10B2C0007047F0B583B001AB6A460C460646FFF7FF
:10B2D000BFFF009905463046FDF7F4FDB4F90C3088
:10B2E000D8B1019A154F0099F76343F08003A38109
:10B2F0002060206161611AB92B43A38103B0F0BDC6
:10B300003046B4F90E1000F0ABFBA0B1A38923F0D6
:10B31000030343F001031BB2EEE79A05EED423F0DA
:10B32000030304F1430243F002030121A3812260DD
:10B3300022616161E2E7B4F90C30DDE76DAA4000FB
:10B3400082B049B15AB16BB113780B601278101CFE
:10B3500018BF012002B0704701A9002AF3D110469E
:10B3600002B070476FF00100F4E700BF002900F061
:10B3700095802DE9F04F0D46164683B0804606F1C4
:10B380000B07FEF7F1F955F804EC162F2EF0030425
:10B39000A5F108093CD810221746BE423DD8944278
:10B3A00043DAC44B996809EB0400884200F0B4808A
:10B3B000436823F0010101444968C9074CD51EF0D8
:10B3C000010F00F09B8031464046FDF77BFD0646AD
:10B3D00000283AD055F8043C23F001034B44A0F177
:10B3E00008029A4200F02181221F242A00F20781DC
:10B3F000132A00F2DB8003462A461168196051685F
:10B40000596092689A6029464046FFF783FC1CE029
:10B4100027F00707002F3A46BFDA00260C233046F4
:10B42000C8F8003003B0BDE8F08F2E46E31B0F2BA9
:10B430001ED8D9F8043003F0010323434C44C9F863
:10B440000430636843F0010363604046FEF792F9FD
:10B45000304603B0BDE8F08F23F00303E1189142BA
:10B460001FDBC36882682E46D3600C469A60DDE716
:10B47000D9F8042009EB070102F001024C4443F023
:10B4800001031743C9F804704B60636843F001037C
:10B49000083163604046FFF73DFCD6E71146FDF7F3
:10B4A00011BD1EF0010F8ED155F8081CA9EB010A41
:10B4B000DAF8041021F003010B442344934225DB06
:10B4C000C26881685646CA609160DAF80C1056F876
:10B4D000080F221F242AC160886000F29480132A7A
:10B4E0006FD92968CAF808106968CAF80C101B2AB5
:10B4F00000F2A28008350AF1100263E055F8083C1A
:10B50000A9EB030ADAF8041021F00301631893424F
:10B51000FFF659AF5646D8E7416821F0030BA34424
:10B5200007F11000834556DA1EF0010F7FF44BAF90
:10B5300055F8081CA9EB010ADAF8041021F0030100
:10B540008B445845E2DC5646DAF80C1056F8080FE2
:10B55000221F242AC160886000F28F80132A40F2E3
:10B560008A802968CAF808106968CAF80C101B2A72
:10B5700000F28A8008350AF11002296811606968B2
:10B580005160A96891600AEB0701ABEB070242F03A
:10B59000010299604A60DAF8043003F001031F43A6
:10B5A0004046CAF80470FEF7E5F851E72B680360DF
:10B5B0006B6843601B2A2DD800F1080305F10802CF
:10B5C0001BE732462968116069685160A96891607B
:10B5D0001C46D1462AE709EB0701ABEB070B4BF002
:10B5E000010299604A6055F8043C03F001031F43CF
:10B5F000404645F8047CFEF7BDF82E4628E729466C
:10B60000FEF700F8FFE6294630461C46D146FDF716
:10B61000F9FF0BE7AB688360EB68C360242A17D09F
:10B6200000F1100305F11002E7E650F8043C23F0A6
:10B6300003031C442E46F9E6A968CAF81010E9680D
:10B64000CAF81410242A0CD010350AF11802B9E7F0
:10B650002B6903616B69436105F1180200F118035E
:10B66000CBE62A69CAF818206A69CAF81C2018357E
:10B670000AF12002A6E732467FE7294630460193C9
:10B68000FDF7C0FF019B7EE7A968CAF81010E968C2
:10B69000CAF81410242A03D010350AF118026CE7F6
:10B6A0002A69CAF818206A69CAF81C2018350AF1F4
:10B6B000200262E73806002010B50C46B1F90E10E2
:10B6C00000F0F6F9002803DB236D0344236510BD69
:10B6D000A38923F48053A38110BD00BF2DE9F0415D
:10B6E0001646B1F90C201F46D3050C46054607D572
:10B6F00000220223B1F90E1000F0C4F9B4F90C20B5
:10B70000B4F90E1022F48052A2813B4632462846FC
:10B71000BDE8F04100F0A4B810B50C46B1F90E1028
:10B7200000F0B0F9A389421C0EBF23F4805343F408
:10B7300080532065A38110BDB1F90E1000F008B947
:10B74000F8B50D461446064610B1836B002B4BD05E
:10B75000B4F90C20A369A36091B2080739D5236915
:10B76000002B36D0EDB289042F4615D522686169C9
:10B77000D31A8B421CDA0133A168501C0139A16035
:10B780002060157062699A421AD0A389DB0701D53F
:10B790000A2D15D03846F8BD616E42F4005221F4EE
:10B7A0000051A281226861666169D31A8B42E2DB93
:10B7B00021463046FFF730F940B922680123DBE724
:10B7C00021463046FFF728F90028E3D04FF0FF3735
:10B7D000E0E721463046FFF70BF80028F6D1B4F930
:10B7E0000C20236991B2BDE7FFF76EF9B0E700BF07
:10B7F000F0B5064685B01F4689B1104C104D24683F
:10B80000646B002C08BF2C46D4F8E040A047431CD2
:10B8100003D100228A233A60336005B0F0BD0C46A4
:10B820000649074A0968496B002908BF11462246A4
:10B83000D1F8E04001A9A047E9E700BF08020020D5
:10B840004C0A002021B1FF2A04D80A700120704759
:10B85000084670478A2303604FF0FF30704700BFEF
:10B8600070B50D46084C114606461A462846002378
:10B870002360FAF729FB431C00D070BD2368002B1E
:10B88000FBD0336070BD00BFB01B00202DE9F84332
:10B890002C4D0646286898460F469146FFF7D4FC83
:10B8A000294B1C68D4F84831002B3ED05A681F2A17
:10B8B0001CDC02F1010E76B103EB82010124C1F818
:10B8C0008890D3F8880194402043022EC3F8880161
:10B8D000C1F8088123D00232C3F804E0286843F895
:10B8E0002270FFF7B3FC0020BDE8F883174B0BB3C1
:10B8F0004FF4C870FDF7D6FA0346D8B1D4F8482102
:10B900000260002141600A46C4F848014FF0010E70
:10B91000C0F88811C0F88C11002EDCD0CCE7D3F829
:10B920008C110C43C3F88C41D5E704F5A673C4F819
:10B930004831BBE72868FFF789FC4FF0FF30BDE8CE
:10B94000F88300BF480A00203CC24000A58E40009A
:10B9500038B5074C0023054608462360FAF7B6FEC3
:10B96000431C00D038BD2368002BFBD02B6038BDB2
:10B97000B01B002070B559B105460C4610B1836B61
:10B98000002B3CD0636ED80705D5B4F90C302BB929
:10B990000026304670BDA38999053CD5214628462E
:10B9A000FEF79AFFE36A064633B1E16928469847F5
:10B9B0000028B8BF4FF0FF36A3891A0622D4216BA6
:10B9C00041B104F14003994202D02846FFF7A2F9A1
:10B9D00000232363616C21B12846FFF79BF9002304
:10B9E0006364FFF79DF8636E0022DB07A2810ED52A
:10B9F000A06DFFF727FCFFF799F8304670BDFFF701
:10BA000063F8BFE721692846FFF784F9D7E7A06DFF
:10BA1000FFF71CFCECE7A06DFFF716FCB4F90C3047
:10BA2000002BBBD1666E16F00106B1D1A06DFFF7F9
:10BA30000DFC304670BD00BF38B50B46074C0546BF
:10BA40001146184600232360FAF743FE431C00D03A
:10BA500038BD2368002BFBD02B6038BDB01B002005
:10BA600038B5074C0023054608462360FAF736FE32
:10BA7000431C00D038BD2368002BFBD02B6038BDA1
:10BA8000B01B002070B50D46084C114606461A46FC
:10BA9000284600232360FAF723FE431C00D070BD24
:10BAA0002368002BFBD0336070BD00BFB01B0020AB
:10BAB00070B50D46084C114606461A462846002326
:10BAC0002360FAF7E7F9431C00D070BD2368002B10
:10BAD000FBD0336070BD00BFB01B002053B94AB922
:10BAE000002908BF00281CBF4FF0FF314FF0FF3086
:10BAF00000F07AB9ADF1080C6DE904CE00F006F85B
:10BB0000DDF804E0DDE9022304B070472DE9F047D9
:10BB10008C460D460446089E002B51D18A4217469A
:10BB20006DD9B2FA82FEBEF1000F0BD0CEF1200C1F
:10BB300001FA0EF520FA0CFC02FA0EF74CEA050C9D
:10BB400000FA0EF44FEA174A250CBCFBFAF81FFA6C
:10BB500087F90AFB18CC45EA0C4508FB09F3AB4210
:10BB60000AD9ED1908F1FF3280F02381AB4240F28F
:10BB70002081A8F102083D44ED1AA4B2B5FBFAF009
:10BB80000AFB105544EA054400FB09F9A14509D90F
:10BB9000E41900F1FF3380F00A81A14540F20781EA
:10BBA00002383C44A4EB090440EA08400021002E7E
:10BBB00061D024FA0EF4002334607360BDE8F0878E
:10BBC0008B4207D9002E54D0002186E82100084678
:10BBD000BDE8F087B3FA83F1002940F08E80AB42D4
:10BBE00002D3824200F2FA80841A65EB0305012039
:10BBF000AC46002E3FD086E81010BDE8F08712B9A1
:10BC00000127B7FBF2F7B7FA87FEBEF1000F34D178
:10BC1000EB1B3A0C1FFA87FC0121B3FBF2F8250C51
:10BC200002FB183345EA03450CFB08F3AB4207D986
:10BC3000ED1908F1FF3002D2AB4200F2D18080460C
:10BC4000ED1AA3B2B5FBF2F002FB105543EA05442E
:10BC50000CFB00FCA44507D9E41900F1FF3302D224
:10BC6000A44500F2B8801846A4EB0C0440EA084052
:10BC70009DE731463046BDE8F087CEF1200405FA55
:10BC80000EF307FA0EF720FA04F83A0C25FA04F43A
:10BC900048EA0308B4FBF2F14FEA184502FB1144ED
:10BCA0001FFA87FC45EA044501FB0CF3AB4200FA9E
:10BCB0000EF409D9ED1901F1FF3080F08A80AB4212
:10BCC00040F2878002393D44EB1A1FFA88F5B3FB36
:10BCD000F2F002FB103345EA034500FB0CF3AB42E4
:10BCE00007D9ED1900F1FF386FD2AB426DD9023898
:10BCF0003D44EB1A40EA01418FE7C1F1200722FAE7
:10BD000007F88B4005FA01F448EA030320FA07FE1E
:10BD10004FEA134CFD404EEA040EB5FBFCF94FEA26
:10BD20001E440CFB19551FFA83F844EA054509FB2C
:10BD300008F4AC4202FA01F200FA01FA08D9ED184F
:10BD400009F1FF3043D2AC4241D9A9F102091D44A7
:10BD50002D1B1FFA8EFEB5FBFCF00CFB10554EEAB6
:10BD6000054400FB08F8A04507D9E41800F1FF35A9
:10BD700029D2A04527D902381C4440EA0940A4EB47
:10BD80000804A0FB02894C45C6464D4615D312D087
:10BD900056B1BAEB0E0364EB050404FA07F7CB4087
:10BDA0001F43CC40376074600021BDE8F08718461F
:10BDB000F8E69046E0E6C245EAD2B8EB020E69EB3F
:10BDC00003050138E4E72846D7E7404691E7814676
:10BDD000BEE7014678E702383C4445E7084608E7F5
:10BDE000A8F102083D442BE7704700BF01000000A6
:10BDF0000200000004000000080000001000000025
:10BE000020000000400000008000000000008000D2
:10BE10000000000100000002000000040000000813
:10BE20000000001000000000000000000000000002
:10BE30000000000000000000000000000000000002
:10BE400000000000000000000000000001280110B8
:10BE50000253290351FF01026902026B10058001A0
:10BE600040401103F0AA1104C00040000AC2010AB8
:10BE7000010A010A0090022D70110000891080074C
:10BE80008003C0078003C003C0020003580020C61F
:10BE900037000D000F00110008180010F0030C20EF
:10BEA00000060B0B3308810256000B0011000882BC
:10BEB0000256000B00110002350002250103F0AA12
:10BEC0001002D10203F0AA110AC2010A010A010AF2
:10BED00000900203FF5A8102650B0EF9585F666DF0
:10BEE000747B828990979EA5AC03F0AA1202D3209E
:10BEF00003BF37BE02038102360003F0AA1104C556
:10BF0000000140000128011002038102532903515E
:10BF1000FF01026900026B102D7011000089108072
:10BF200009F004F804F804F804F80200041B0020E7
:10BF300091BF0011000F00190009180010F0030C48
:10BF40002000060B0B330580013E3E11088101E104
:10BF50000010001000088201E1001000100002250E
:10BF60000103F0AA1002D10203F0AA110AC2010AC9
:10BF7000010A010A00900203F0AA1202D32003BFB3
:10BF800007BE03FF5A8102650B0EF9585F666D7498
:10BF90007B828990979EA5AC00000000FF00FF0007
:10BFA00056585230300000005553415254000000A2
:10BFB0004661696C656420746F20637265617465A5
:10BFC000207573617274207461736B0D0A00000038
:10BFD00000FFFFFFFFFFFF0009273412D20400001B
:10BFE000021E0104A5000078E70000000000000028
:10BFF0000000000000000101010101010101010137
:10C00000010101010101000000000000000000002A
:10C010000000FFFF0000001800000000000000000A
:10C020000000000000000000000000000000000010
:10C03000000000000000000000000000000000FC04
:10C04000004265796F6E6400000000000000010D81
:10C05000702079000022092839540F80DF137F00F7
:10C060003F801F00EF0917000E8001001EF50A0037
:10C07000FF0EFF003F801F007F071B000E800100A6
:10C080007E00073A029281000800000000000000D4
:10C0900000000000000000000000000000000000A0
:10C0A0000000000000000000000000000000000090
:10C0B0000000000000000000000000000000000080
:10C0C0000000000000000000000000000000F890E8
:10C0D0005265706F727400004661696C656420740B
:10C0E0006F206372656174652048494420726570F1
:10C0F0006F7274207461736B0D0A00004932430043
:10C100004661696C656420746F2063726561746553
:10C1100020493243207461736B0D0A0054494D4528
:10C12000445F5354415254004661696C6564207405
:10C130006F206372656174652074696D6564207336
:10C14000746172747570207461736B0D0A00000065
:10C15000414443004661696C656420746F206372DA
:10C160006561746520414443207461736B0D0A005E
:10C1700049444C450000000000C20100C00000001E
:10C1800000080000000000002D2D20467265657239
:10C19000746F73204578616D706C65202D2D0A0DCC
:10C1A00000000000444953504C4159424F41524411
:10C1B0002056302E342E31002D2D2025730A0D00EF
:10C1C00031323A30393A3439000000004F6374207C
:10C1D00020372032303232002D2D20436F6D7069B0
:10C1E0006C65643A202573202573202D2D0A0D00DF
:10C1F0005553424C6F6164004661696C65642074FC
:10C200006F2063726561746520555342204C6F61E5
:10C21000646572207461736B0D0A0000737461634E
:10C220006B206F766572666C6F772025782025739A
:10C230000D0A00006C6F676600000000100200200D
:10C24000303132333435363738394142434445464C
:10C25000000000003031323334353637383961620E
:10C260006364656600000000286E756C6C29000030
:10C2700020202020202020202020202020202020BE
:10C2800030303030303030303030303030303030AE
:10C2900043000000504F5349580000002E0000009A
:10C2A0000020202020202020202028282828282086
:10C2B000202020202020202020202020202020207E
:10C2C00020881010101010101010101010101010E6
:10C2D00010040404040404040404041010101010D6
:10C2E00010104141414141410101010101010101A0
:10C2F00001010101010101010101010110101010F2
:10C300001010424242424242020202020202020271
:10C3100002020202020202020202020210101010C5
:10C3200020000000000000000000000000000000ED
:10C3300000000000000000000000000000000000FD
:10C3400000000000000000000000000000000000ED
:10C3500000000000000000000000000000000000DD
:10C3600000000000000000000000000000000000CD
:10C3700000000000000000000000000000000000BD
:10C3800000000000000000000000000000000000AD
:10C39000000000000000000000000000000000009D
:10C3A00000000000F8B500BFF8BC08BC9E4670470E
:10C3B000B9A840006D014000F8B500BFF8BC08BC4A
:08C3C0009E4670474901400050
:08C3C80044F7FF7F01000000B3
:10C3D00030B482B0049C5BB31D46036843F48033E1
:10C3E0000360C9B241F0B441416083680193019B8D
:10C3F00013F0010FF9D1002306E0990001F5800147
:10C40000096845F823100133A342F6D3D2B242F0B3
:10C41000B442426083680193019B13F0010FF9D08D
:10C42000036823F480330360002002B030BC7047FF
:10C430000220FAE70160704782B04160836801938F
:10C44000019B13F0010FF9D0019800F00E0002B02B
:10C450007047FFFFFFFF0000DD024000E1024000E7
:10C46000E3024000E7024000EB02400025034000E9
:10C4700075034000ED024000F1024000FD02400063
:10C480000147470150010020C000002000000000CB
:10C49000C80000206401002009028500030100C0DB
:10C4A00032080B0002010100020904000000010132
:10C4B000000209240100011E0001010C24020101F7
:10C4C0000200020300000009240302010100010030
:10C4D0000904010000010200020904010101010236
:10C4E0000002072401020101000B240201020210D4
:10C4F0000180BB000905840500010100000725013A
:10C5000000000000090402000103000000092111DD
:10C5100001000122260007058103400004000000FD
:10C520001201000200000040BD35010100010102BE
:10C5300000010000880000209C0000207001002005
:10C54000CD324000ED32400045334000EF32400034
:10C550000000000006FFFF0901A1010902090315FF
:10C560000026FF007508954081020906090715009D
:10C5700026FF0075089540B102C0000000030000CE
:10C5800000000000000000000000000000000000AB
:10C59000000000000000000000000000000000009B
:10C5A00000000000000000000403090447656E65F8
:10C5B000726963005553422053746572656F204D54
:10C5C0006963726F70686F6E6500010000127A0017
:10C5D000AAAAAAAA01000000100200200000000080
:10C5E00000000000FC04002064050020CC050020B1
:10C5F000000000000000000000000000000000003B
:10C60000000000000000000000000000000000002A
:10C61000000000000000000000000000000000001A
:10C62000000000000000000000000000000000000A
:10C6300000000000000000000000000000000000FA
:10C6400000000000000000000000000000000000EA
:10C6500000000000000000000000000000000000DA
:10C6600000000000000000000000000000000000CA
:10C6700000000000000000000000000000000000BA
:10C6800000000000000000000100000000000000A9
:10C690000E33CDAB34126DE6ECDE05000B0000006E
:10C6A000000000000000000000000000000000008A
:10C6B000000000000000000000000000000000007A
:10C6C000000000000000000000000000000000006A
:10C6D000000000000000000000000000000000005A
:10CA1000380600203806002040060020400600208E
:10CA2000480600204806002050060020500600203E
:10CA300058060020580600206006002060060020EE
:10CA4000680600206806002070060020700600209E
:10CA5000780600207806002080060020800600204E
:10CA600088060020880600209006002090060020FE
:10CA70009806002098060020A0060020A0060020AE
:10CA8000A8060020A8060020B0060020B00600205E
:10CA9000B8060020B8060020C0060020C00600200E
:10CAA000C8060020C8060020D0060020D0060020BE
:10CAB000D8060020D8060020E0060020E00600206E
:10CAC000E8060020E8060020F0060020F00600201E
:10CAD000F8060020F80600200007002000070020CC
:10CAE000080700200807002010070020100700207A
:10CAF000180700201807002020070020200700202A
:10CB000028070020280700203007002030070020D9
:10CB10003807002038070020400700204007002089
:10CB20004807002048070020500700205007002039
:10CB300058070020580700206007002060070020E9
:10CB40006807002068070020700700207007002099
:10CB50007807002078070020800700208007002049
:10CB600088070020880700209007002090070020F9
:10CB70009807002098070020A0070020A0070020A9
:10CB8000A8070020A8070020B0070020B007002059
:10CB9000B8070020B8070020C0070020C007002009
:10CBA000C8070020C8070020D0070020D0070020B9
:10CBB000D8070020D8070020E0070020E007002069
:10CBC000E8070020E8070020F0070020F007002019
:10CBD000F8070020F80700200008002000080020C7
:10CBE0000808002008080020100800201008002075
:10CBF0001808002018080020200800202008002025
:10CC000028080020280800203008002030080020D4
:10CC10003808002038080020400800204008002084
:10CC20004808002048080020500800205008002034
:10CC300058080020580800206008002060080020E4
:10CC40006808002068080020700800207008002094
:10CC50007808002078080020800800208008002044
:10CC600088080020880800209008002090080020F4
:10CC70009808002098080020A0080020A0080020A4
:10CC8000A8080020A8080020B0080020B008002054
:10CC9000B8080020B8080020C0080020C008002004
:10CCA000C8080020C8080020D0080020D0080020B4
:10CCB000D8080020D8080020E0080020E008002064
:10CCC000E8080020E8080020F0080020F008002014
:10CCD000F8080020F80800200009002000090020C2
:10CCE0000809002008090020100900201009002070
:10CCF0001809002018090020200900202009002020
:10CD000028090020280900203009002030090020CF
:10CD1000380900203809002040090020400900207F
:10CD2000480900204809002050090020500900202F
:10CD300058090020580900206009002060090020DF
:10CD4000680900206809002070090020700900208F
:10CD5000780900207809002080090020800900203F
:10CD600088090020880900209009002090090020EF
:10CD70009809002098090020A0090020A00900209F
:10CD8000A8090020A8090020B0090020B00900204F
:10CD9000B8090020B8090020C0090020C0090020FF
:10CDA000C8090020C8090020D0090020D0090020AF
:10CDB000D8090020D8090020E0090020E00900205F
:10CDC000E8090020E8090020F0090020F00900200F
:10CDD000F8090020F8090020000A0020000A0020BD
:10CDE000080A0020080A0020100A0020100A00206B
:10CDF000180A0020180A0020200A0020200A00201B
:10CE0000280A0020280A0020300A0020300A0020CA
:10CE1000FFFFFFFF000002008C1B0020430000000A
:10CE20000000000000000000000000000000000002
:10CE300000000000000000000000000043000000AF
:10CE400000000000000000000000000000000000E2
:10CE5000000000000000000000000000430000008F
:10CE600000000000000000000000000000000000C2
:10CE7000000000000000000000000000430000006F
:10CE800000000000000000000000000000000000A2
:10CE9000000000000000000000000000430000004F
:10CEA0000000000000000000000000000000000082
:10CEB000000000000000000000000000430000002F
:10CEC0000000000000000000000000000000000062
:10CED000000000000000000000000000430000000F
:10CEE0000000000000000000000000000000000042
:10CEF00000000000000000000000000045B84000F5
:10CF000041B3400000000000A0C240009CC24000AD
:10CF1000A0C14000A0C14000A0C14000A0C140008D
:10CF2000A0C14000A0C14000A0C14000A0C140007D
:10CF3000A0C14000FFFFFFFFFFFFFFFFFFFFFFFF5C
:10CF4000FFFF000001004153434949000000000079
:10CF500000000000000000000000000000000000D1
:10CF60000000000000004153434949000000000058
:10CF700000000000000000000000000000000000B1
:08CF80000000000000000000A9
:0400000500406465EE
:00000001FF
